:105C76007584008534D28535D37584018536D28501
:105C860037D31260EA12612412615EE4F535F53409
:105C960030007C300662856582856483E55A601033
:105CA600E0F535855AF0A4F53485F035A3A38008D0
:105CB600E0F535A3E0F534A3858265858364E56563
:105CC6006567700CE5646566700675650075640247
:105CD600856382856283E539F0A3E538F0A3858282
:105CE60063858362E56365677025E5626566701F97
:105CF6007563007562028017E55A600DE539855AAD
:105D0600F0A4F53485F0358006853834853935308C
:105D1600010CE534253AF534E535353BF5353002E9
:105D260010E52A8528F0A42534F534E5F03535F557
:105D360035300310E50A852DF0A42534F534E5F059
:105D46003535F535300410E511852CF0A42534F5EC
:105D560034E5F03535F535E4F537F53630097A3082
:105D66000560856582856483E55B600EE0855BF092
:105D7600A4F53685F037A3A38008E0F537A3E0F550
:105D860036A3858265858364E5656567700CE56481
:105D96006566700675650075640285638285628333
:0E5DA600E53BF0A3E53AF0A3858263858362B6
:105DB400E56365677025E5626566701F7563007548
:105DC40062028017E55B600DE53B855BF0A4F53668
:105DD40085F0378006853A36853B37300822E55909
:105DE4006012E5398559F0A42536F536E5F03537E6
:105DF400F537800CE5362538F536E5373539F5378E
:105E0400300A10E52A8528F0A42536F536E5F03564
:105E140037F537E537C395324003853237300B10F9
:105E2400E50A852DF0A42536F536E5F03537F53746
:105E3400300C10E511852CF0A42536F536E5F03547
:105E440037F537300D10E518852BF0A42536F536D7
:105E5400E5F03537F537300E10E54E8530F0A425E2
:105E640036F536E5F03537F537E537C39533400376
:105E740085333722905F1A301503125E943016036F
:105E8400125EA4301803125F0A301703125EC72291
:105E9400E50B2509F50BE50C3508F50C93F50A22FD
:105EA400E512250EF512E513350DF51393C313F81A
:105EB400E5142510F514E515350FF51593C31328CE
:105EC400F51122102E08202F3C3032238026D22FA9
:105ED40020300E30312FC22FC232D230754D0080A7
:065EE40024203121C22F31
:105EEA00D232C230754D00801690601A80039060DD
:105EFA0062E54D93F54E054DE54DB44802D22F2289
:105F0A00E5192517F519E51A3516F51A93F5182224
:105F1A007F8285888C8F9295989B9EA1A4A7AAAD13
:105F2A00B0B3B6B9BBBEC1C3C6C9CBCED0D3D5D721
:105F3A00D9DCDEE0E2E4E6E7E9EBEDEEF0F1F2F4DB
:105F4A00F5F6F7F8F9FAFBFCFCFDFDFEFEFEFEFE97
:105F5A00FEFEFEFEFEFDFDFCFCFBFAFAF9F8F7F682
:105F6A00F4F3F2F0EFEDECEAE8E7E5E3E1DFDDDB9D
:105F7A00D8D6D4D1CFCDCAC8C5C2C0BDBAB7B4B2BB
:105F8A00AFACA9A6A3A09D9A9794908D8A87848185
:105F9A007E7A7774716E6B6865625F5C595653508E
:105FAA004D4A4744423F3C393734322F2D2A28265E
:105FBA0024211F1D1B1918161412110F0E0C0B0A7F
:105FCA00080706050404030202010100000000009C
:105FDA000000000000010102020304050607080987
:105FEA000A0B0D0E1011131516181A1C1E20222446
:105FFA0027292B2E303335383A3D404245484B4EFF
:10600A00515456595C606366696C6F7275787B7F10
:10601A00FEFEFEFEFDFCFCFBFAF8F7F6F4F3F1EFE8
:10602A00EDEBE9E7E4E2DFDCDAD7D4D0CDCAC6C3C8
:10603A00BFBCB8B4B0ACA8A39F9B96928D89847F4D
:10604A007A75706B66615C57514C47413C37312C0D
:10605A0026211B16100B050000050B10161C212704
:10606A002C32373D42484D53585D62686D72777CD9
:10607A0081858A8F94989DA1A5AAAEB2B6BABEC1EF
:10608A00C5C8CCCFD2D5D8DBDEE1E3E6E8EBEDEF4D
:10609A00F1F2F4F6F7F8F9FBFBFCFDFEFEFEFEFE5C
:1060AA00000C1926333F4C5864707B86919CA6AF2E
:1060BA00B8C1C9D1D8DEE4EAEFF3F6F9FCFDFEFE79
:1060CA00FEFDFCFAF7F4F0EBE6E0DAD4CCC5BCB49A
:1060DA00ABA1978D83786D61554A3D3125180C0027
:1060EA00E52EF5F0B4010122753A00E53BC394565A
:1060FA004013A4F5F0C394565007E5F02456F53B37
:10610A0022753BAC227456953BA4F8C394565006AC
:10611A00745698F53B22753B0022E52FF5F0B40141
:10612A000122753800E539C394564013A4F5F0C32B
:10613A0094565007E5F02456F539227539AC227485
:10614A00569539A4F8C394565006745698F53922D0
:10615A007539002285452AE529F5F0B4010122E5C1
:10616A002AC394864013A4F5F0C394865007E5F039
:10617A002486F52A22752AFF227486952AA4F8C352
:0E618A0094865006748698F52A22752A002203
:10694100D2F4C2F5C2F675840F85F0C8127258747C
:106951000312699012724C740312699012722F1211
:10696100722F740312699012722F740212699012BD
:10697100722F74281269FC74061269FC740E126974
:10698100FC74011269FC12724C74801269FC22C001
:1069910000A2E092F3A2E192F2A2E292F1A2E392CA
:1069A100F0D2F475840F85F0C8C2F47830D8FE8532
:1069B100F0C87830D8FED00022C00075840FA2E460
:1069C10092F3A2E592F2A2E692F1A2E792F0D2F45A
:1069D10085F0C8C2F47830D8FE85F0C87830D8FE8A
:1069E100D00022EF75840FD2F5C2F685F0C8126986
:1069F100BA12722F12699012722F2275840FC2F58A
:106A0100C2F685F0C81269BA12722F126990127219
:106A11002F22EF14A2E492E6C2E4D2E71269FC222B
:106A2100740F1269FC22740D1269FC227F01126A33
:106A31001378107F201269E4D8F9227F11126A13AA
:106A410078107F201269E4D8F9227F01126A137845
:106A5100207F201269E4D8F922C0077F018004C099
:106A6100077F11126A13D007C082C083C007EF7578
:106A7100F010906A8B1272707810E493FF1269E43F
:096A8100A3D8F7D007D083D0821E
:106A8A0022202020202020202020202020202020FA
:106A9A002057414954494E4720464F522052494EA9
:106AAA00472054454C434F20414E53574552454485
:106ABA0020205741495420464F5220444953434FBE
:106ACA002020205445535420204641494C45442017
:106ADA0020202054455354202050415353454420EC
:106AEA00202020454550524F4D20544553542020D4
:106AFA0020204155582052454C4159205445535461
:106B0A002020205055534820544F2054414C4B20AC
:106B1A002054455354203320434841522F53554261
:106B2A002054455354204649584544205354524909
:106B3A004E544553542056415249422053545249C7
:106B4A004E464143544F52592044454641554C54B0
:106B5A002050524F4752414D4D494E47204D4F44C8
:106B6A004553494D504C455820524550454154458E
:106B7A00522020205245434F5244494E472020205C
:016B8A0020EA
:08000300027DBC0000000000BA
:08000B00027DBD0000000000B1
:08001300027F1D000000000047
:08001B003200000000000000AB
:09002300320000000000000000A2
:08002B00027DC000000000008E
:08003300320000000000000093
:0A003B003200000000000000000089
:0900430032000000000000000082
:08004B0032000000000000007B
:08005300320000000000000073
:08005B00027E250000000000F8
:08006300320000000000000063
:08006B00027E440000000000C9
:08007300027DC6000000000040
:08007B00027F1E0000000000DE
:08008300027E1F0000000000D6
:08008B0032000000000000003B
:10009300027F3C00000000000000000000000000A0
:1000A3003275FF0775FFDE75FFAD75840F75E107C8
:1000B30075E20475E34475840F75A43575A5097558
:1000C300A6FF75A7FF759CFF759D00759E00759F24
:1000D300F075D8FF75E8FF75F80F75AD0F758401DE
:1000E30075893075888F75840275893075888F7529
:1000F300840F758A80758C67780874FF0000000090
:100103000000000000000000D5E0F1D8EDE58C30E0
:10011300E7FB759701758A0043890475840075B7F9
:100123001075840F438901758D01758F01758E02DA
:100133007480D5E0FD438902E58930E4FB759702BD
:1001430075840075D10775840075BB0175BA007598
:10015300BCF075C70075C60075C5FF75C4FF75E8AB
:100163008175840275BB0475BA0075BCF175C60050
:1001730075C4FF75E88875840075D484758401752A
:10018300D484758400C2F8759A47759D1A43F8099B
:1001930075870075840075B90075A90075910075A0
:1001A300985075840175981075840075C04075C3A7
:1001B3000075CFC9758400758E0075892075880513
:1001C300758400758A00758B6F758CF4758D6F431C
:1001D300885075840075C90075CA0075CB0075CC4D
:1001E3000075CD0075840175C91875CA8075CBFB80
:1001F30075CDFB75CC80D2CA75840275C91875CAD2
:10020300A675CBAF75CDAF75CCA6D2CA7584007574
:10021300EF0275A8AF75B80075E6A475E71775F614
:100223000075F7019000007F007E20E4F0A3DFFC5F
:02023300DEFAF1
:100235007528FF752BFF752CFF752DFF7531FF7523
:1002450032FF7533FF751D0A751E0A751F06752762
:020255000A227B
:107DBC0032C28D32758400C2CF32C0E0C083C08223
:107DCC00C0D0C000C0F0C2CFB21A201A23125C7609
:107DDC00151BE51B7009751B0A7584017588AF1599
:107DEC001CE51C7009751C607584027588AF8011C8
:107DFC00125E78153CE53C7008753C04758400D225
:107E0C008B758400D2ECD0F0D000D0D0D082D0834F
:107E1C00D0E032C2CF027BE132C0E0C0D0C007C09C
:107E2C0000C083C08212861175888FD082D083D017
:107E3C0000D007D0D0D0E032C0E0C0D0C000C083AA
:107E4C00C082C08420122875840F30DF3CE5E854D2
:107E5C000F240283801044313233343536373839AD
:107E6C00302A23414243F546D2127547C8801A1571
:107E7C0047E5477006E546D2E7F54675840F20DFE7
:107E8C0008C212D211D22BD21D20142975840F30A6
:107E9C00F83DE5E854F0C4240283801044313233B9
:107EAC00343536373839302A23414243F548D21419
:107EBC007549C8801A1549E5497006E548D2E7F5B9
:107ECC004875840F20F808C214D213D22AD21C127F
:107EDC00865E151DE51D702A751D0A1286AB151ED2
:107EEC00E51E701E751E0A128736151FE51F7012CF
:107EFC00751F061287771527E527700675270A1256
:107F0C008788D084C28DD082D083D000D0D0D0E0EE
:057F1C00323220100DBF
:107F2100D21085BF3B85BE3A75BB01800BC210855F
:107F3100BF3985BE3875BB00C2ED32C0E0C0D0E5A7
:107F41004AB4000A054A85BE4575BB07803DB401A8
:107F51000A054A85BE4275BB048030B4020A054A4F
:107F610085BE4575BB068023B4030A054A85BE4319
:107F710075BB048016B4040A054A85BE4575BB0568
:107F81008009754A0085BE4475BB04C2EDD0D0D0CE
:027F9100E032DC
:106B8B00202020434F532041435449564520202079
:106B9B000020524144494F205349474E414C494EE6
:106BAB00470020202052494E47204F55542020208B
:106BBB002020002020414E535745522050484F4E25
:106BCB0045202000204E4F2050484F4E45204C4929
:106BDB004E4520200054454C434F204F52494749C6
:106BEB004E415445200020494E50555420434150AE
:106BFB0020434F44452000494E50555420414343B8
:106C0B00455353434F4445004155544F20414E5338
:106C1B005745522050414745002020504147494E8F
:106C2B0047204D4F44452020200020204D4F4E49FA
:106C3B00544F52204D4F44452020002020202053FC
:106C4B0054414E4442592020202020524144494F68
:106C5B00204F524947494E4154452054454C434FD0
:106C6B00204F524947494E4154452053494D504CB2
:106C7B00455820524543204D4F444553494D504CA8
:106C8B00455820584D54204D4F4445202020444911
:106C9B0053434F4E4E45435420202020202044493F
:106CAB00414C20544F4E452020202020202042557F
:106CBB00535920544F4E4520202020204E4F205614
:106CCB004F582054494D454F55542020414354496A
:106CDB005654592054494D455220202020204C49D0
:106CEB004E452043555420202020202054494D450B
:106CFB004F55542054494D455220202020204454B8
:106D0B004D4620524144494F2020202020204454FE
:106D1B004D462054454C434F20202054414C4B4270
:106D2B0041434B2054494D454F555454454C434FCB
:106D3B00204449414C20544F4E4520494E50555408
:106D4B002050484F4E45204E554D42205054542014
:106D5B00444953434F4E4E4543542052494E4720CE
:106D6B004355544F46462054494D4548414C4620C7
:106D7B004455504C4558205245434548414C4620BC
:106D8B004455504C4558205854524D2020204655C0
:106D9B004C4C204455504C455820202050484F4EC9
:106DAB00452054494D454F55542020204D4F4249C5
:0B6DBB004C452054494D454F555420D5
:109EB10012C77C75840F1200A412DE2612E3AF12C2
:109EC1006A2D20A5031256F1E49000E9F012F18AFF
:109ED1005005E49000E9F012DBDB12EAF912762F6B
:109EE100900172E07006900174E0600612F228128F
:109EF100D73820A40512DE7480F820A60A12D9AC46
:109F0100E49000E9F080EB301C10C21C90009F74BB
:109F110001F09000ABF09000FEF0301D10C21D90DA
:109F210000A07401F09000A5F09000FDF09000E910
:109F3100E0B4150050BC909F3EF8282873029F7D25
:109F4100029F83029F89029F8F029F95029F9B021E
:109F51009FA1029FA7029FAD029FB3029FB9029FDB
:109F6100BF029FC5029FCB029FD1029FD7029FDDF7
:109F7100029FE3029FE9029FEF029FF512A3BF0236
:109F81009EF3126198029EF312B319029EF312AB73
:109F9100B5029EF3128146029EF3127817029EF3D8
:109FA10012E531029EF312E9AE029EF312E3F102D1
:109FB1009EF312E6D0029EF312D7A2029EF312EF95
:109FC10081029EF312C9D8029EF312847D029EF390
:109FD10012B756029EF31279FD029EF312B5B10239
:109FE1009EF312D2F3029EF312DF54029EF312CDBE
:0A9FF100E4029EF312A99E029EF303
:10A3BF0012EE7312F15A12F0B612F16612F14D123B
:10A3CF00F14612F1F512F1EF12F21F12F1E312F151
:10A3DF00E912F22512F1D712F1DD12F20712F20D86
:10A3EF0012F1D112F21312F1CB12F22B12F22890BA
:10A3FF000172E07006900174E0600612F22812D725
:10A40F0038E49001C3F0A3F0900081F0900080F049
:10A41F009000D5F09000CAF09000CEF09000CFF0F1
:10A42F009000C6F09000D9F09000DDF09000E1F0C0
:10A43F00900095F090009AF090009EF09000AAF096
:10A44F009000A3F09000BEF0900097F090009974E8
:10A45F0037F0E49000CDF09000D3F09000D4F0905E
:10A46F0000C8F09000D8F09000DCF09000E0F09081
:10A47F0000E4F090009DF09000A2F09000A9F09001
:10A48F0000C1F09000A0F090009FF09000A5F09018
:10A49F0000ABF09000FEF09000FDF09001BBF0904B
:10A4AF0001BEF090019EF09001A1F09000A67420E3
:10A4BF00F09000A7F09001B77401F0A3F0A3F0A300
:10A4CF00F09001C2F0E49001C1F012EE8D7BFF7AA3
:10A4DF006C794612E952126A3C900122E0F52F90F6
:0CA4EF000123E0F52E9000E9E004F022CB
:1061980012EFB712BC0E12A88112B14C900137E071
:1061A8006009900132E0600312EE21900166E06020
:1061B800229000D8E0B4011B9000FC741EF0E4901B
:1061C80000D3F09000D4F09000CAF09000CFF09087
:1061D80000CEF09000FCE0700612B4D912A28190B3
:1061E8000174E0700302627D9000FEE070030262B9
:1061F8007DE4F0E5486423706012D43F5077900046
:10620800D8E0600E12EFB77BFF7A6B798B12E952F8
:1062180080EC9001BE7401F012F1CB12EE5912F02D
:10622800357BFF7A6B799C12E952900171E0B401D9
:106238000312F15412E4F31270019001BCE06007FC
:106248009000E97413F02212F04112EE73E4900109
:10625800A3F09001A2F00265829001B8E09001B726
:10626800F09001B9E09001B8F09001BAE09001B95E
:10627800F0A3E548F012F0A59000D4E0607812F1A0
:10628800CB7BFF7A6B79AD12E952E49000D4F090A1
:1062980001A104F012EE5912F035900171E0B40139
:1062A8000312F15412F035900169E070149001184E
:1062B800E0F52C12EFD712F1E612F10612F1E9809F
:1062C80018900169E0755E00F55F12E4F390018AA9
:1062D8007430F012700112F0A512F04112EE7390B2
:1062E8000171E0B4010312F15A900132E0FF60033A
:1062F800B4010312F1D19000A2E070030264389057
:1063080000A9E060030264389000A2F012F1CB907B
:1063180001A1E0640160030263A912EE5912F0358D
:10632800900171E0B4010312F15412F035E49001C8
:10633800A1F0900134E0FF900098F0900161E090A6
:106348000094F09000E7EFF0900157E09000C2F061
:10635800900158E09000C3F0900183E09001BFF0F5
:10636800900184E09001C0F0900132E0700312E8DF
:106378004E900132E0B4010312ECF8900132E0B41F
:10638800020312EF06E49000A5F09000E97405F00E
:1063980012F0AE900171E0640260030265EA02F156
:1063A8005412F18A5046900186E0604012EE59126C
:1063B800F03512F06412726412725812725812F1A7
:1063C8004612726412F06412726412725812725891
:1063D80012F14612726412F0641272641272581248
:1063E800725812F146127264E402658212F0AE909D
:1063F8000171E0B4020312F154753DC89000A17414
:106408006EF09000AC7464F0E4F55CE55C2481FF08
:10641800E433FE7D2012C94E055CE55CC394104050
:10642800EAE490019AF0753E969000E97403F02230
:106438009000A9E0700302650512F18A50469001A8
:1064480086E0604012EE5912F03512F06412726460
:1064580012725812725812F14612726412F06412D3
:10646800726412725812725812F14612726412F063
:106478006412726412725812725812F146127264DF
:10648800E402658212F1CB7BFF7A6C795612E952ED
:10649800900182E0602E12EE5912F035900171E001
:1064A800B4010312F154E4F54F900182E0F55090E5
:1064B8000120E0F528E49000A5F012F1D49000E95D
:1064C8007412F022E49000A9F09000BEF09000C190
:1064D800F09000BDF012E7E49000ADE0B4200712A0
:1064E800EBABE402658212F0AE900171E0B40203F6
:1064F80012F154753E969000E97406F02290009DC2
:10650800E0602D7BFF7A6C795612E952E490009D89
:10651800F09000A904F09000A8F0900181E0FF70CD
:10652800030265EA90019E7401F09000C5EFF02225
:10653800302C2312EC2CC22C12DBDB12EAF9127677
:106548002F900172E07006900174E0600612F22844
:1065580012D738E4802430202612E77812DBDB12C9
:10656800EAF912762F900172E07006900174E060EB
:106578000612F22812D738C220E49000E9F02290DF
:1065880000D3E0605D12F1CB7BFF7A6B79BE12E934
:106598005212F0AE900171E0B4020312F154E4908B
:1065A80000D3F09000CEF0753DC87BFF7A6C796619
:1065B80012E952753F96753DC8900170E0FF60136F
:1065C800E4F54F8F50900121E0F52812F1DAE4F557
:1065D8003E8009754F0B753E3C12F0599000E974E6
:0365E80002F0229C
:10B31900E53D600302F21F12F196501612F19050AA
:10B32900117BFF7A6B79CF12E95212F11612F0FEF6
:10B339008034E53ED39401400312F21CE53EB4018A
:10B349000612F146E4F53EE53ED39401400302B30B
:10B35900FAE53F7002806812A4FB12BC0E12C59375
:10B369009000C8E06003E480561282FE4004753FF5
:10B37900962212F1DD302C2312EC2C12DBDB12EABF
:10B38900F912762F900172E07006900174E0600660
:10B3990012F22812D738C22CE4802430202612E772
:10B3A9007812DBDB12EAF912762F900172E070064F
:10B3B900900174E0600612F22812D738C220E49096
:10B3C90000E9F02290017CE0600C9000E97410F033
:10B3D900E49000A2F02290016FE0FF7002800CEF70
:10B3E900B4010E9000A2E06008E4F09000E974084E
:02B3F900F02240
:10ABB50012AE8CE53D600302ACAF12F1965018124F
:10ABC500F19050137BFF7A6B79CF12E95212F1168F
:10ABD50012F0FEE402AC88E53E602512EE597BFFDB
:10ABE5007A6D793612E952900132E0700312F21350
:10ABF50012F1CE9000A1746EF09000AC7464F02256
:10AC05007BFF7A6D794612E952900132E0700D12A0
:10AC1500EE73900171E0B4010312F15A900132E034
:10AC2500FF6003B4010312F1D190009FE06042E49C
:10AC3500F012F2139000C1E07070900199E548F0B0
:10AC45009000C17401F09000A17428F09000AC74DC
:10AC550064F090019AE0FF04F0EF2481FFE433FEF5
:10AC6500AD4812C94E90019AE0D3940F403CE4F0F0
:10AC7500229000C1E0600612F21312EA3E9000AC89
:10AC8500E070059000E9F0229000A1E070107BFFD4
:10AC95007A6C795612E9529000E9740CF022900012
:0BACA500C8E060069000E9740AF0228D
:1081460012EFB7128C1712CC6A12CBEA12BC0E12BF
:10815600E74012EBD712BCCA12AE8C12A13E12A493
:10816600FB12EB5312EE0412EB7F12EA6E12A88199
:1081760090009DE0600DE4F09000C804F09000EAE5
:10818600740BF090019EE060199000C5E0701090AD
:1081960000C804F09000EA740CF0E490019EF0121E
:1081A600DCE2900132E0B4020E12E32BEF6005121E
:1081B600F210800312F213900176E0600C9001BD7C
:1081C600E0700612F20712F1EF900132E07034907F
:1081D6000185E0600A9001C2E0640170268021906A
:1081E60000E0E0701E90017DE0601512F1D112F200
:1081F6002812F06412725812725812F14612726402
:1082060002E84E900132E06401702A12E32BEF601F
:108216002490017DE0601B12F1D112F22890011228
:10822600E0F52D12F06412725812725812F14612CD
:10823600726402ECF8900132E06402702412E32BBF
:10824600EF601E90017DE0601512F1D112F2281246
:10825600F06412725812725812F14612726402EFEA
:1082660006302C3412EE7312F15A12F16612F0B681
:1082760012EC2C12DBDB12EAF912762F900172E077
:108286007006900174E0600612F22812D738C22CEC
:1082960012F1F512F1D1803230203512EE7312F15F
:1082A6005A12F16612F1EF12F1D112E77812DBDB06
:1082B60012EAF912762F900172E07006900174E0CE
:1082C600600612F22812D738C220E49000E9F022A4
:0D82D6009000C8E060069000E9740AF022F4
:1078170012EFB7128C1712CC6A12BC0E12E7401285
:10782700BCCA12AE8C12A13E12A4FB12EB5312EE8D
:107837000412EB7F12EA6E12A88190009DE0600DA2
:10784700E4F09000C804F09000EA740BF090019EF9
:10785700E060199000C5E070109000C804F0900037
:10786700EA740CF0E490019EF012DCE290018AE0E9
:10787700B431119000C4E0700B9000C804F0900080
:10788700EA7408F0900176E0600C9001BDE07006A4
:1078970012F20712F1EF12E32BEF6015900132E0BD
:1078A700B40109900136E0700312F1C812F210809A
:1078B7000612F1CB12F2139001C1E0B4011090014E
:1078C70032E0700A900185E0B4010302795A12EFA1
:1078D70093EF600C900132E07006900185E0600C38
:1078E70012E32BEF6014900132E0600EE49000E0A9
:1078F700F09000DDF090019B04F012EF93EF700C15
:10790700900132E07006900185E0600C12E32BEFE6
:10791700704E900132E0604890019BE06026900134
:1079270065E06020900113E0F52D12F059127258AE
:1079370012725812725812725812725812F146E4A3
:1079470090019BF012CBEA9000E0E06013900132C7
:10795700E0700302E91B900132E0B4010302ED85F8
:1079670012F19C500F12F213AF4812F06F9000E91A
:107977007407F022302C3712EE7312F15A12F166A7
:1079870012F0B612F21312EC2C12DBDB12EAF91228
:10799700762F900172E07006900174E0600612F293
:1079A7002812D73812F1EF12F213C22C803530208B
:1079B7003812EE7312F15A12F16612F1EF12F1D189
:1079C70012F21312E77812DBDB12EAF912762F9024
:1079D7000172E07006900174E0600612F22812D777
:1079E70038C220E49000E9F0229000C8E0600690D9
:0679F70000E9740AF02211
:10E53100E53E703812F196501A12F19050157BFF9A
:10E541007A6B79CF12E95212F11612F0FEE49000C3
:10E55100E9F02212EA0E9000C1E06010E4F012EE40
:0DE56100599000E9740CF0E49000BDF02228
:10E9AE0012A4FB9000C8E06006E49000E9F0221289
:10E9BE00F19C401B12F14D12F21090017CE0900080
:10E9CE00E960097410F0E49000A2F0227405F022C0
:10E3F10090015DE0FF64026005EF6403702CE4F5B9
:10E401004F90015CE0F550900120E0F52812F1D425
:10E4110012F1DA12EE5912F035900171E0B40103F4
:10E4210012F1549000E9E004F0229000E9740FF039
:01E4310022C8
:10E6D00012A4FB1282FE502F12F1D712F1DD12F0BC
:10E6E00041900132E0700D12EE73900171E0B401BF
:10E6F0000312F15A900132E0FF6003B4010312F1FA
:08E70000D19000E9740FF02232
:10D7A2007BFF7A6C799612E9529000EAE075F010EC
:10D7B200A424A6F9746C35F0FA7BFF12E983900178
:10D7C2005DE0FF64016005EF6403703012F2131232
:10D7D200F1D1E4F54F90015CE0F550900120E0F5C5
:10D7E2002812F1D412F1DA12EE5912F035900171C9
:10D7F200E0B4010312F154E4F53E8006753E64750F
:09D802004F0B9000E9E004F02254
:10EF8100E53E700D1282FE5008E49000E9F012F0A7
:02EF910041221B
:10C9D800E53E600302CA6012F210900132E0700D69
:10C9E80012EE73900171E0B4010312F15A90013212
:10C9F800E0FF6003B4010312F1D1900134E0FF902D
:10CA08000098F0900161E0900094F09000E7EFF05A
:10CA1800900157E09000C2F0900158E09000C3F0F8
:10CA2800900183E09001BFF0900184E09001C0F094
:10CA3800900132E0700312E84E900132E0B4010335
:10CA480012ECF8900132E0B4020312EF06E4900011
:09CA5800A5F09000E97405F0223C
:10847D007BFF7A6B79E012E9527BFF7A6B79F1120F
:10848D00E9839000FDE060199000FBE0FF04F074BB
:10849D00EB2FF582E43400F583E546F0E49000FD22
:1084AD00F0900175E0FF9000FBE06F600302860421
:1084BD0012D8DD40030285F812EE5912F035900105
:1084CD0071E0B4010312F15412F03512E4F312709D
:1084DD00019001BCE060079000E97413F02212F0E6
:1084ED0041900132E0700D12EE73900171E0B40114
:1084FD000312F15A12E14C90018AE0FFB4300302ED
:10850D00860BEF6431705D900173E09000C4F090C4
:10851D000134E0FF900098F0900161E0900094F03C
:10852D009000E7EFF0900157E09000C2F0900158F5
:10853D00E09000C3F0900183E09001BFF0900184C2
:10854D00E09001C0F0900132E0700312E84E90010E
:10855D0032E0B4010312ECF8900132E0B4020312E0
:10856D00EF06805B90018AE06432705F900134E029
:10857D00FF900098F0900161E0900094F09000E77A
:10858D00EFF0900157E09000C2F0900158E090009C
:10859D00C3F0900183E09001BFF0900184E0900161
:1085AD00C0F0900132E0700312E84E900132E0B459
:1085BD00010312ECF8900132E0B4020312EF06E46D
:1085CD009000A5F09000E97405F02290018AE0B4C6
:1085DD003325E490009EF090017BE09000A1F0E443
:1085ED009000A2F09000E9740EF02212EE3EE4909D
:1085FD0000FBF0753F6422E53F700812F09BE4909C
:04860D0000E9F0226E
:10B756007BFF7A6C790212E98312B3FB9000A2E0B8
:10B766006061E4F0900134E0FF900098F090016190
:10B77600E0900094F09000E7EFF0900157E0900021
:10B78600C2F0900158E09000C3F0900183E0900170
:10B79600BFF0900184E09001C0F0900132E07003A8
:10B7A60012E84E900132E0B4010312ECF890013237
:10B7B600E0B4020312EF06E49000A5F09000E974ED
:10B7C60005F02212A4FB12BC0E9000C8E0600280B5
:10B7D60048302C2212EC2C12DBDB12EAF912762FFF
:10B7E600900172E07006900174E0600612F2281271
:10B7F600D738C22C802330202512E77812DBDB12E3
:10B80600EAF912762F900172E07006900174E060FA
:0FB816000612F22812D738C220E49000E9F0227F
:1079FD00E53E6003027BE090016BE060447BFF7A23
:107A0D006C791312E95212EE5912F035900171E0B2
:107A1D00B4010312F15412F03590016BE0755E0064
:107A2D00F55F12E4F312700112F041900132E07033
:107A3D001012EE73900171E0B4010312F15A12F1BC
:107A4D00D1900172E0B4011C7BFF7A6C792412E9AC
:107A5D0052E49000FBF0753F649000FDF09000E95A
:107A6D00740DF02212F21012F1D190016BE070033F
:107A7D00027B6F90018AE0FFB43006E49000E9F0DC
:107A8D0022EF6431705E900173E09000C4F09001BC
:107A9D0034E0FF900098F0900161E0900094F09038
:107AAD0000E7EFF0900157E09000C2F0900158E030
:107ABD009000C3F0900183E09001BFF0900184E04D
:107ACD009001C0F0900132E0700312E84E90013247
:107ADD00E0B4010312ECF8900132E0B4020312EFAE
:107AED0006027BD590018AE064327056900134E035
:107AFD00FF900098F0900161E0900094F09000E705
:107B0D00EFF0900157E09000C2F0900158E0900026
:107B1D00C3F0900183E09001BFF0900184E09001EB
:107B2D00C0F0900132E0700312E84E900132E0B4E3
:107B3D00010312ECF8900132E0B4020312EF0602D9
:107B4D007BD590018AE0B43319E490009EF090014A
:107B5D007BE09000A1F0E49000A2F09000E9740E9B
:107B6D00F02212EE5912F035900171E0B4010312BA
:107B7D00F15412F035900134E0FF900098F090012F
:107B8D0061E0900094F09000E7EFF0900157E090E5
:107B9D0000C2F0900158E09000C3F0900183E09096
:107BAD0001BFF0900184E09001C0F0900132E070CF
:107BBD000312E84E900132E0B4010312ECF890018B
:107BCD0032E0B4020312EF06E49000A5F09000E954
:047BDD007405F02219
:10B5B1007BFF7A6C793512E98312B9C312BC0E1282
:10B5C100BCCA12AE8C12A13E12A4FB12F1F512F10B
:10B5D100EF12E32BEF600512F210800312F2131247
:10B5E100F19C500F12F213AF4812F06F9000E97402
:10B5F10007F022302C3712EE7312F15A12F1661253
:10B60100F0B612F21312EC2C12DBDB12EAF912760D
:10B611002F900172E07006900174E0600612F2282A
:10B6210012D73812F1EF12F213C22C8035302038C4
:10B6310012EE7312F15A12F16612F1EF12F1D112F8
:10B64100F21312E77812DBDB12EAF912762F90017E
:10B6510072E07006900174E0600612F22812D73889
:10B66100C220E49000E9F0229000C8E06007900059
:10B67100E9740AF0229000A2E0B40108E4F090001D
:05B68100E97411F02244
:10D2F30012EE59900171E0B4010312F15412F035AA
:10D30300900134E0FF900098F0900161E090009468
:10D31300F09000E7EFF0900157E09000C2F0900129
:10D3230058E09000C3F0900183E09001BFF09001BA
:10D3330084E09001C0F0900132E0700312E84E9057
:10D343000132E0B4010312ECF8900132E0B40203BD
:0FD3530012EF06E49000A5F09000E97405F022B7
:10DF54001282FE504312F1D712F04112EE73E49094
:10DF640000A9F09000BEF09000C1F09000BDF01246
:10DF7400E7E49000ADE0B4200912EBABE49000E9D3
:10DF8400F02212F0AE900171E0B4020312F1547564
:09DF94003E969000E97406F022AB
:10CDE400900192E06430702F12F05912F06412F046
:10CDF400EE12F14612F0DE9001BCE014F0E0705B3C
:10CE04009001BEE06002803F9000E97414F090014C
:10CE140076E09001BDF022900118E0F52C12EFD7D6
:10CE240012F1E612F0FE12F0FE12F0FE12F1E91217
:10CE3400F10612F10612F1069001BCE014F0E07064
:10CE44001A9001BEE06006E49000E9F022900176B9
:0CCE5400E09001BDF09000E97414F022A1
:10A99E0012F041900132E0700D12EE73900171E0F1
:10A9AE00B4010312F15A12E14C90018AE0FFB43067
:10A9BE0006E49000E9F022EF6431705D900173E0DF
:10A9CE009000C4F0900134E0FF900098F090016187
:10A9DE00E0900094F09000E7EFF0900157E09000C7
:10A9EE00C2F0900158E09000C3F0900183E0900116
:10A9FE00BFF0900184E09001C0F0900132E070034E
:10AA0E0012E84E900132E0B4010312ECF8900132DC
:10AA1E00E0B4020312EF06805B90018AE0643270AC
:10AA2E005F900134E0FF900098F0900161E090009B
:10AA3E0094F09000E7EFF0900157E09000C2F09094
:10AA4E000158E09000C3F0900183E09001BFF090B8
:10AA5E000184E09001C0F0900132E0700312E84EE4
:10AA6E00900132E0B4010312ECF8900132E0B4022E
:10AA7E000312EF06E49000A5F09000E97405F022B1
:10AA8E0090018AE0B43318E490009EF090017BE0D0
:10AA9E009000A1F0E49000A2F09000E9740EF02274
:10E91B007BFF7A6C798612E98312E14C12F21312A7
:10E92B00F1CE12EE5912F035900171E0B4010312E1
:10E93B00F154900161E0900094F09000E97404F0C0
:01E94B0022A9
:10E84E007BFF7A6C797612E98312E32BEF60051267
:10E85E00F210800312F21312F1D112F22812F041CB
:10E86E0012EE73900171E0B4010312F15A9000E9B7
:04E87E007405F0220B
:10ED85007BFF7A6D798612E98312E14C12F2131238
:10ED9500F1CE900161E0900094F09000E97404F0E8
:01EDA500224B
:10ECF8007BFF7A6D797612E98312E32BEF600512B8
:10ED0800F210800312F21312F1D112F2289000E9E6
:04ED18007405F0226C
:10EF06007BFF7A6D799612E98312F1CE12E14C906D
:06EF160000E97405F02281
:10ED630020202020202052494E47202020202020F0
:10ED73000020202020205354414E4442592020207B
:02ED830020006E
:10B4D9009000CAE0FFEF701190016EE0FF9000CC80
:10B4E900EFF09000CAE004F0229000CAE0FFEFB448
:10B4F900012412F18440159000CB7464F07BFF7A2B
:10B50900ED796312E9529000CAE004F07BFF7AED0D
:10B51900797412E952229000CAE0FFEF6402704781
:10B5290012F18450429000CBE0FFEF600B9000CB0A
:10B53900E0FFEFD3945A40069000CAE4F02290004D
:10B54900CCE014F09000CCE0FFEF701B90016DE0AF
:10B55900FFEF70069000CD7401F09000CAE004F08E
:10B569009000CB74C8F0229000CAE0FFEF6403702A
:10B57900369000CBE0FFEF701490016DE0FFEF60B3
:10B58900069000CD7401F09000CAE4F02212F18413
:10B5990040159000CB74C8F07BFF7AED796312E90E
:08B5A90052229000CAE4F022D6
:10A281009000CEE0FFEFD3940140059000CEE4F0C2
:10A291009000CFE0FFEFD3940340059000CFE4F0AE
:10A2A1009000CDE0FFEF70139000D0E0FFEF700B56
:10A2B1009000CEE4F09000CFE4F0229000CDE0FFDA
:10A2C100EF700322800F9000CDE4F090016CE0FF6D
:10A2D1009000D0EFF09000CEE0FFEF701890016A8F
:10A2E100E0FFEF601090016AE0FF9000D1EFF09085
:10A2F10000CEE004F09000CEE0FFEFB4011C90012D
:10A301006AE0FFEF60149000D1E014F09000D1E01A
:10A31100FFEF70069000D37401F09000CFE0FFEFE3
:10A321007018900167E0FFEF6010900167E0FF9007
:10A3310000D2EFF09000CFE004F09000CFE0FFEF0B
:10A34100B40123900167E0FFEF601B9000D2E0149D
:10A35100F09000D2E0FFEF700D9000D47401F09006
:10A3610000CFE004F0229000CFE0FFEF64027030F4
:10A37100900167E0FFEF6028900168E0FFEF603D2A
:10A38100900168E0FFEFB401079000CFE004F022F4
:10A39100900168E0FFEFB402079000D47401F0224D
:10A3A1009000CFE0FFEFB40314900167E0FFEF608E
:0EA3B1000C9000D47401F09000CFE014F02264
:10A4FB009000C6E0FFEF701E12F196500812F1901B
:10A50B00500302A636900163E0FF9000C9EFF09074
:10A51B0000C6E004F0229000C6E0FFEF640170403B
:10A52B009000C9E0FFEF600302A63612F1964012CD
:10A53B0012F190500D9000C77401F09000C6E0042A
:10A54B00F02212F190500302A63612F1964003024C
:10A55B00A6369000C77402F09000C6E004F02222E9
:10A56B009000C6E0FFEF6402600302A60090016258
:10A57B00E0FFEF700302A636900162E0FFEFB4013B
:10A58B002212F190400302A63612F196400302A666
:10A59B0036900164E0FF900198EFF09000C67403D1
:10A5AB00F02222900162E0FFEF640270489000C736
:10A5BB00E0FFEFB4011B12F190401612F19650110F
:10A5CB009000C87401F09000EA7404F09000C6E4A7
:10A5DB00F09000C7E0FFEFB4021B12F19640161289
:10A5EB00F19050119000C87401F09000EA7404F0DF
:10A5FB009000C6E4F09000C6E0FFEF6403702C906F
:10A60B000162E0FFEFB40123900198E0FFEF701BB4
:10A61B0012F190501612F19650119000C87401F07F
:0CA62B009000EA7404F09000C6E4F022F5
:108A9F009000D5E0FFEF7052900126E0FFEF6026C7
:108AAF00900127E0FFE544D39F4013900128E0FF9A
:108ABF009000D7EFF09000D5E004F022802C9000CA
:108ACF00D8E4F0228024900127E0FFE544C39F50B3
:108ADF0013900128E0FF9000D7EFF09000D57403BA
:108AEF00F02280069000D8E4F0229000D5E0FFEF4E
:108AFF0064017039900127E0FFEF24FBFFE544D3B9
:108B0F009F40239000D7E0FFEF6003028C16900088
:108B1F00D87401F0900129E0FF9000D6EFF090009B
:108B2F00D5E004F022229000D5E4F022229000D567
:108B3F00E0FFEF64027031900127E0FFEF24FBFFAD
:108B4F00E544D39F400B900129E0FF9000D6EFF052
:108B5F00229000D6E0FFEF6003028C169000D8E45D
:108B6F00F09000D5E4F022229000D5E0FFEF6403EF
:108B7F007047900127E0FF7E00EF2405FFEE3400E1
:108B8F00FEAD447C00C3ED9FEE6480F8EC648098EA
:108B9F0050209000D7E0FFEF706D9000D87401F077
:108BAF00900129E0FF9000D6EFF09000D5E004F09F
:108BBF0022229000D5E4F022229000D5E0FFEF644E
:108BCF0004703F900127E0FF7E00EF2405FFEE3495
:108BDF0000FEAD447C00C3ED9FEE6480F8EC648032
:108BEF0098500B900129E0FF9000D6EFF0229000F3
:108BFF00D6E0FFEF70119000D8E4F09000D5E4F0CC
:088C0F0022229000D5E4F022BE
:10CB6A009000D5E0FFEF701612F16C407290012828
:10CB7A00E0FF9000D7EFF09000D5E004F02290009B
:10CB8A00D5E0FFEF6401702C12F16C40219000D7C0
:10CB9A00E0FFEF701F9000D87401F0900129E0FFC8
:10CBAA009000D6EFF09000D5E004F02280069000C5
:10CBBA00D5E4F0229000D5E0FFEFB4022212F16C26
:10CBCA00400B900129E0FF9000D6EFF0229000D6AA
:10CBDA00E0FFEF700A9000D8E4F09000D5E4F0226C
:10EFB700900125E0FFEF600412CB6A22128A9F229C
:108C17009000D9E0FFEF705290012AE0FFEF602645
:108C270090012BE0FFE543D39F401390012CE0FF19
:108C37009000DBEFF09000D9E004F022802C900048
:108C4700DCE4F022802490012BE0FFE543C39F5032
:108C57001390012CE0FF9000DBEFF09000D9740334
:108C6700F02280069000DCE4F0229000D9E0FFEFCC
:108C77006401703690012BE0FFEF24FBFFE543D33F
:108C87009F40219000DBE0FFEF701F9000DC740134
:108C9700F090012DE0FF9000DAEFF09000D9E004AA
:108CA700F02280069000D9E4F0229000D9E0FFEF8F
:108CB700B4022D90012BE0FFEF24FBFFE543D39F88
:108CC700400B90012DE0FF9000DAEFF0229000DAE0
:108CD700E0FFEF700B9000DCE4F09000D9E4F022A5
:108CE7009000D9E0FFEF6403704790012BE0FF7E0F
:108CF70000EF2405FFEE3400FEAD437C00C3ED9F7B
:108D0700EE6480F8EC64809850219000DBE0FFEF80
:108D1700701F9000DC7401F090012DE0FF9000DAE5
:108D2700EFF09000D9E004F02280069000D9E4F03B
:108D3700229000D9E0FFEF6404703E90012BE0FF22
:108D47007E00EF2405FFEE3400FEAD437C00C3ED4B
:108D57009FEE6480F8EC648098500B90012DE0FF43
:108D67009000DAEFF0229000DAE0FFEF700B90004E
:0F8D7700DCE4F09000D9E4F0229000D9E4F0227F
:10CBEA009000DDE0FFEF701612F17850729001307C
:10CBFA00E0FF9000DFEFF09000DDE004F02290000B
:10CC0A00DDE0FFEF6401702C12F17850219000DF13
:10CC1A00E0FFEF701F9000E07401F0900131E0FF37
:10CC2A009000DEEFF09000DDE004F0228006900034
:10CC3A00DDE4F0229000DDE0FFEFB4022212F17889
:10CC4A00500B900131E0FF9000DEEFF0229000DE01
:10CC5A00E0FFEF700A9000E0E4F09000DDE4F022DB
:10CC6A009000E1E0FFEF701612F172507290012EFF
:10CC7A00E0FF9000E3EFF09000E1E004F022900082
:10CC8A00E1E0FFEF6401702C12F17250219000E391
:10CC9A00E0FFEF701F9000E47401F090012FE0FFB5
:10CCAA009000E2EFF09000E1E004F02280069000AC
:10CCBA00E1E4F0229000E1E0FFEFB4022212F17207
:10CCCA00500B90012FE0FF9000E2EFF0229000E27B
:10CCDA00E0FFEF700A9000E4E4F09000E1E4F02253
:10EF9300900133E0FFEF60069000E4E0FF2212E30C
:02EFA3002B221F
:10E32B00900125E0FFEF600D12F16C40047F01803E
:10E33B00027F002222900126E0FFEF60139001275D
:10E34B00E0FFE544D39F40047F0122227F0022227D
:10E35B00900127E0FFE544C39F50047F0122227FF9
:02E36B0000228E
:10CAE600535155452020434F53202053454E53451F
:10CAF600004F4E20202020202020202020202020F3
:10CB060020004F46462020202020202020202020C4
:10CB160020200044544D46204445434F444520546C
:10CB260045535400191823A01296203D129623A0AF
:10CB3600129627631488203D148823A0148827633F
:10CB460016B8203D16B823A016B827631918203D3D
:10CB56001918276312962B8C14882B8C16B82B8CDD
:04CB660019182B8CE3
:10C77C0012F1AA12F1A712F16CE433F55C12F1ADCF
:10C78C00E433F55C12F1B0E433F55C12F1B3E4334D
:10C79C00F55C12F1B6E433F55C12F1B9E433F55CF7
:10C7AC0012F1BCE433F55C12F1BFE433F55C12F129
:10C7BC00C2E433F55C12F17EE433F55C12F1C5E4AE
:10C7CC0033F55C12F18AE433F55C12F1C812F1CB4B
:10C7DC0012F1D412F1D712F1DA12F1DD12F1E012EA
:10C7EC00F1E312F1E612F1E912F20412F20712F27D
:10C7FC000A12F20D12F21612F21912F21C12F21F98
:0CC80C0012F22212F22512E19102F22B2E
:06F1540075840FD2FC22BD
:06F15A0075840FC2FC22C7
:06F1600075840FD2B722F6
:06F1660075840FC2B72200
:08F0AE0075840FD2FED21F226F
:08F0B60075840FC2FEC21F2287
:10EE590075840FD2FD900171E0B4010312F1549051
:0AEE69000187E0B4010312F16022FA
:10EE730075840FC2FD900171E0B4010312F15A9041
:0AEE83000187E0B4010312F16622DA
:03F1A700C29322EE
:03F1AA00D29322DB
:06F16C0075840FA2FA22D7
:03F1AD00A2A022FB
:03F1B000A2A122F7
:03F1B300A2A222F3
:03F1B600A2A322EF
:03F1B900A2A422EB
:03F1BC00A2A522E7
:03F1BF00A2A622E3
:03F1C200A2A722DF
:06F1720075840FA2F922D2
:06F1780075840FA2DD22E8
:06F17E0075840FA2DE22E1
:03F1C500A29222F1
:06F1840075840FA2DA22DF
:06F18A0075840FA2DB22D8
:06F1900075840FA2D822D5
:06F1960075840FA2D922CE
:06F19C0075840FA2F822A9
:03F1C800D2082248
:03F1CB00C2082255
:03F1CE00D2092241
:03F1D100C209224E
:03F1D400D20A223A
:03F1D700C20A2247
:03F1DA00D202223C
:03F1DD00C2022249
:03F1E000D20B222D
:03F1E300C20B223A
:03F1E600D20C2226
:03F1E900C20C2233
:03F1EC00D20D221F
:03F1EF00C20D222C
:03F1F200D218220E
:03F1F500C218221B
:03F1F800D215220B
:03F1FB00C2152218
:03F1FE00D2162204
:03F20100C2162210
:03F20400D20E2205
:03F20700C20E2212
:03F20A00D20F22FE
:03F20D00C20F220B
:03F21000D2002207
:03F21300C2002214
:03F21600D2012200
:03F21900C201220D
:03F21C00D20322F8
:03F21F00C2032205
:03F22200D20422F1
:03F22500C20422FE
:10E14C00E4FDFCED25E0FFEC33FE74002FF582744A
:10E15C00023EF583E4F0A3F00DBD00010CBC0EE310
:10E16C00BDE0E07562027563007402F564F56590BC
:10E17C000135E075F0BEA4AEF02400F567EE340274
:04E18C00F566D2055D
:01E19000226C
:03F22800C20522FA
:10E19100E4FDFCED25E0FFEC33FE74002FF5827405
:10E1A100023EF583E4F0A3F00DBD00010CBC0EE3CB
:10E1B100BDE0E07562027563007402F564F5659077
:10E1C1000135E075F0BEA4AEF02400F567EE34022F
:04E1D100F566D20617
:01E1D5002227
:03F22B00C20622F6
:0BF0590075081575095ED215D2032260
:0BF0640075081575095ED215D20B224D
:07F14600C215C203C20B2237
:0BF06F00900110128D86D216D20422F0
:0BF07A00900111128D86D216D20C22DC
:0C8D8600E0F52CE4F512F513F514F515DA
:108D9200EF12AB8F8E8D238E7C2A8DCA308DDC3103
:108DA2008DEE328E00338E12348E24358E36368E10
:108DB20048378E5A388E6B398E9E418EAF428EC0A6
:108DC200438ED14400008EE990CB2AE493F50D74D2
:108DD2000193F50E90CB2C028EE090CB2EE493F50E
:108DE2000D740193F50E90CB30028EE090CB32E4FD
:108DF20093F50D740193F50E90CB34028EE090CB77
:108E020036E493F50D740193F50E90CB38028EE0A3
:108E120090CB3AE493F50D740193F50E90CB3C029E
:108E22008EE090CB3EE493F50D740193F50E90CB5A
:108E320040028EE090CB42E493F50D740193F50E5F
:108E420090CB44028EE090CB46E493F50D740193EF
:108E5200F50E90CB48028EE090CB4AE493F50D7468
:108E62000193F50E90CB4C807590CB4EE493F50DAB
:108E7200740193F50E90CB50806490CB52E493F53D
:108E82000D740193F50E90CB54805390CB56E4931E
:108E9200F50D740193F50E90CB58804290CB5AE4B5
:108EA20093F50D740193F50E90CB5C803190CB5EFF
:108EB200E493F50D740193F50E90CB60802090CB76
:108EC20062E493F50D740193F50E90CB64800F90DC
:108ED200CB66E493F50D740193F50E90CB68E493A1
:088EE200F50F740193F5102255
:07F14D00C216C20CC204222D
:0FEFD700750D0C750ECD750F0B7510BCD2162273
:09F0A500C217C20EC218C20D22EE
:10D9AC007BFF7ACA79E612E95212F16C7BFF4006D2
:10D9BC007ACA79F780047ACB790812E9837F171237
:10D9CC006A13AF441272B590006FE0FF1269E490D5
:10D9DC000070E0FF1269E4900071E0FF1269E47FCF
:10D9EC001C126A13AF431272B590006FE0FF1269FC
:10D9FC00E4900070E0FF1269E4900071E0FF0269AE
:01DA0C00E435
:0BF0850075081A7509ABD215D20B22DA
:0BF090007508027509ABD215D20B22E7
:10DE74009001C3E0701D7BFF7ACB791912E952122D
:10DE84006A3C9001C37401F0E49000E9F012F11EC1
:10DE9400126A2D9001C3E0B40120302A0DC22AE594
:10DEA40048547F900090F012D211302B0DC22BE514
:0BDEB40046547F90008FF012CE6022D9
:10443F00202020202020202020202020202020206D
:10444F00202020202020202020202020202020205D
:10445F002054454C434F2050524F4752414D20203E
:10446F0020524144494F2050524F4752414D202036
:10447F002050484F4E452050524F4752414D20201B
:10448F0020434F4D50552050524F4752414D202001
:10449F00202041434345535320434F444520202080
:1044AF0044544D462054454C434F204C4556454CA3
:1044BF0044544D4620524144494F204C4556454C9B
:1044CF004245455020524144494F204C4556454C9A
:1044DF00424545502054454C434F204C4556454C82
:1044EF004357494420524144494F204C4556454C6F
:1044FF0054454C434F20524144494F204C45564C54
:10450F00524144494F2054454C434F204C45564C43
:10451F00524144494F204C494D4954204C45564C2B
:10452F002020504147494E47204C4556454C2020AE
:10453F00435443535320524144494F204C45564C0A
:10454F0044435320524144494F204C4556454C203B
:10455F004C545220524144494F204C4556454C2013
:10456F002020524550454154204C4556454C202063
:10457F002045494120544F4E45204C4556454C202F
:10458F004C4F57204755415244204C4556454C20DF
:10459F0048494748204755415244204C4556454CC1
:1045AF00564F494345205241444930204C45564CC3
:1045BF00564F4943452054454C434F204C45564C8C
:1045CF00202020524144494F204741494E2020206E
:1045DF0020202054454C434F204741494E20202056
:1045EF00202020564F494345204741494E20202047
:1045FF0020434F53204F5220535155454C43482091
:10460F002020434F5320504F4C41524954592020A2
:10461F00434F53205452494747455220564F4C540D
:10462F00434F5320414351554953542054494D450D
:10463F00434F532052454C454153452054494D4516
:10464F002053454E534520504F4C41524954592009
:10465F0053454E205452494747455220564F4C54CC
:10466F0053454E20414351554953542054494D45CC
:10467F0053454E2052454C454153452054494D45D5
:10468F005220564F582041435155495354494F4E8C
:10469F0020525820564F582052454C4541534520E3
:1046AF005420564F582041435155495354494F4E6A
:1046BF0020545820564F582052454C4541534520C1
:1046CF00204F5045524154494E47204D4F444520AD
:1046DF0020564F58204F52204341525249455220A5
:1046EF002020564F582041435449564954592020B1
:1046FF00202054454C434F2044454C415920202005
:10470F002050524956414359204D4F4445202020B7
:10471F002052455045415420454E41424C452020A2
:10472F00202020204944204D4F4445202020202088
:10473F002043574944204F5220564F49434520208C
:10474F0020435749442043414C4C205349474E2066
:10475F002043574944204652455155454E43592011
:10476F002020494420494E54455256414C20202088
:10477F0020525054522048414E472054494D452015
:10478F0020525054522041435449564954592020E5
:10479F00205250545220434F5552544553592020C4
:1047AF002042454550204652455155454E435920CC
:1047BF002020434F4E4E45435420434F4445202025
:1047CF00444953434F4E4E45435420434F44452095
:1047DF0020204143434553532044454C4159202009
:1047EF002041435449564954592054494D4552206C
:1047FF002054494D454F55542054494D4552202082
:10480F002020505454204155544F4449414C2020AE
:10481F00505454204D494E494D554D2054494D4506
:10482F00505454204D4158494D554D2054494D45F4
:10483F0020202053544154494F4E204944202020DA
:10484F00202020204944204D4F4445202020202067
:10485F00204255535920444953434F4E4E454354DC
:10486F004255535920444953434F204359434C45D4
:10487F004449414C20544F4E4520444953434F2007
:10488F004449414C20444953434F2054494D4520FE
:10489F00204C494E4520444953434F4E4E454354B7
:1048AF002020204C494E452044454C415920202082
:1048BF004C494E4520494E41435449564554592081
:1048CF005420434F5552544553592042454550208B
:1048DF0042555359204348414E4E454C204D4F4E63
:1048EF002052494E474F5554204E554D4245522068
:1048FF00202052494E474F5554204D4F44452020BC
:10490F002052494E474F555420414C455254202078
:10491F00414E535745522052494E47204E4D425219
:10492F00414E535745522050414745204E4D42521C
:10493F0020202052494E47205350414345202020EC
:10494F00202052494E4720414E5357455220202098
:10495F0052494E47205452414E534954494F4E539A
:10496F0020202052454D4F54452042415345202091
:10497F00414E53572020564F494345204E4D4252EA
:10498F00204155582052454C4159204D4F44452008
:10499F0020202050414745204D4F444520202020C6
:1049AF002054414C4B204241434B2054494D45200C
:1049BF004D4F4220544F204D4F42205041474520EC
:1049CF00204F5645524449414C204449474954537E
:1049DF0043544353532F4443532054494D4552207E
:1049EF002020204245455020414C45525420202044
:1049FF005245504541542053455155454E4345204E
:104A0F00205455524E204F4E2044454C41592020A2
:104A1F00205455524E204F46462044454C41592074
:104A2F002044544D4620434841522054494D45207F
:104A3F0020204D4F4E49544F52204D4F444520207A
:104A4F005220434F5552544553592042454550200B
:104A5F0052454C415920414343455353434F4445DD
:104A6F0052494E47204355544F46462054494D45D1
:104A7F005350454544204449414C20564F494345E6
:104A8F00202050484F4E452054494D454F555420F6
:104A9F00204D4F42494C452054494D454F555420C8
:104AAF00204D414E55414C20434F4E54524F4C20B8
:104ABF004C494E4520425553592044455445435483
:104ACF0020202020202020202020202020202020D7
:104ADF0020202020202020202020202020202020C7
:104AEF0020202020202020202020202020202020B7
:104AFF00202020202020202020202020313D454E26
:104B0F002020202020202020202020524154494FB7
:104B1F002020202020202020202020303D434F53D4
:104B2F002020202020202020202020313D504F53B6
:104B3F0020202020202020202020202031204D53F5
:104B4F0020202020202020202020203130204D53D5
:104B5F0020202020202020202020313030204D53B5
:104B6F0020202020202020202020202020534543BB
:104B7F00202020202020202020202020204D494EA2
:104B8F002020202020202020202020204D4F444571
:104B9F002020202020202020202020313D564F583B
:104BAF00202020202020202020202052494E475313
:104BBF00202020202020202020204359434C4553E3
:104BCF0020202020202020202020313D544F4E45F2
:104BDF002020202020202020204D5347204E554DAF
:104BEF0020202020202020202020434C49434B53BD
:104BFF002020202020202020202020204741494E07
:104C0F002020202020202020303D424541434F4E80
:104C1F0020202020202020202020202046524551D7
:104C2F00202020202020202050414745204E554D48
:104C3F002020202020202020202044494749545361
:104C4F002020202020202020202020424545505386
:104C5F00202020202020202020202020544F4E458F
:104C6F0082010011026C15000182010111036C1504
:104C7F00000182010211046C15000182010311056C
:104C8F006C15000178060411060119000082030A51
:104C9F0011076D1500FF82030B11086D1500FF82C0
:104CAF00030C11096D1500FF82030D110A6D15001C
:104CBF00FF82030E110B6D1500FF82030F110C6D98
:104CCF001500FF820310110D6D1500FF82031111E6
:104CDF000E6D1500FF820312110F6D1500FF820379
:104CEF001311106D1500FF82031411116D1500FFC4
:104CFF0082031511126D1500FF82031611136D1526
:104D0F0000FF82031711146D1500FF820318111590
:104D1F006D1500FF82031911166D1500FF82031A1E
:104D2F0011176D1500FF82031B11186D1500FF82FF
:104D3F00021C11197C15011082021D111A7C15011C
:104D4F001082011E111B7C15011082011F111C6E98
:104D5F00150001820120111D6F1500018203211121
:104D6F001E6D1500FF820222111F70150063820253
:104D7F002311207115006382012411216F15000189
:104D8F0082032511226D1500FF8202261123701553
:104D9F0000638202271124711500638202281125F6
:104DAF007015006382022911267215006382022A90
:104DBF0011277015006382022B1128721500638270
:104DCF00012C11297515000282012D112A7615006B
:104DDF000182022E112B7415006382022F112C7188
:104DEF00150028820130112D6C150001820131113F
:104DFF002E6C150001820132112F7D1500018201E9
:104E0F0033113075150008BE0A341131011100003D
:104E1F0082023E11327E15011482023F1133741546
:104E2F000063820240113472150063820241113512
:104E3F007315006382014211366C15000182024323
:104E4F0011377E1501146E06441138011900006EDA
:104E5F00064A113901190000820250113A72150ADF
:104E6F00638C0251113B73150A63820252113C7419
:104E7F00150063820153113D7B1503098202541102
:104E8F003E72150563820255113F7215056382014B
:104E9F005611407A1500078201571141751500030D
:104EAF0082015811426C1500018201591143781586
:104EBF00020982015A11446C15000182025B1145EF
:104ECF007215146382015C11467515000282025D32
:104EDF0011477115006382025E11487015006382DD
:104EEF00015F11496C150001820160114A6C1500B8
:104EFF0001820161114B77150009820162114C7516
:104F0F00150002820163114D7A150063820164114D
:104F1F004E77150009820265114F7F1500638202DB
:104F2F0066115072150063820167115175150001EA
:104F3F008203681152781501FF82016911537515AB
:104F4F00000182016A11547A15000782016B115515
:104F5F007515000482016C11567515000182026DE2
:104F6F0011577315036382016E11586C150001827E
:104F7F00016F115980150104820270115A731500C7
:104F8F0063820171115B81150009820172115C78D6
:104F9F00150109820373115D711500FF82027411EF
:104FAF005E71150063820275115F721505638201D0
:104FBF007611607515000182017711616C15000182
:104FCF0078037811620119000082027B1163731557
:104FDF00006382017C11647A15000782027D1165DE
:104FEF007315006382027E11667315006382017F61
:104FFF0011676C15000182018011686C150001208A
:10500F00202020202020202020202020202020822F
:10501F00010111020C15000120202020202020204A
:10502F00202020202020202082010111020C1500B9
:10503F000120202020202020202020202020202080
:10504F0020640100110209150001202020202020DA
:10505F002020202020202020202020202020202041
:10506F002020202020202020202054454C4550482F
:10507F004F4E45204E554D424552B410001102017E
:10508F001100002020202020202020202020202060
:10509F002020202020202020202020202020202001
:1050AF002020202020504147494E47204E554D4249
:1050BF00455220AA100011020111000020202020CB
:1050CF00202020202020202020202020010101014D
:1050DF0001010101010000000000000000000000BC
:1050EF0000000000000000000000000000000000B1
:1050FF0000000000000000000000000000000000A1
:10510F000000000000000000000000000000000090
:10511F000000000000000000000000000000000080
:10512F000000000000002020202020202020202030
:10513F0020202020202082010011021E15000101D5
:10514F00010101313233343536FF32323232FFFF53
:10515F00FFFFFFFFFFFF323232FFFF0101010001AE
:10516F0080000A0180000A000A000A0001002801DD
:10517F000000002020202020202020202005141EA9
:10518F001E01052020202020202020202020201E4E
:10519F001E0300050F000101070146016305000012
:1051AF00010100020063000A000000001801030063
:1051BF0006010A0A3200003738392D0000000000BE
:1051CF000000002020202020202020202020202030
:1051DF0020202020202020202020202020202020C0
:1051EF00202020000036333036373036393437310F
:1051FF003937343437373037393738323538353443
:10520F003838353931353934383937343130303140
:10521F00303331303731313031313431313831325F
:10522F003331323731333131333631343131343642
:10523F003135313135363135393136323136353127
:10524F003637313731313733313737313739313805
:10525F0033313836313839313932313936313939EC
:10526F003230333230363231303231383232353209
:10527F0032393233333234313235303235343030F3
:10528F0036303037303135303137303231303233EC
:10529F0030323530323630333130333230333630DE
:1052AF0034333034373035303035313035333035C5
:1052BF0034303635303731303732303733303734AA
:1052CF0031313431313531313631323231323531AC
:1052DF00333131333231333431343131343331349A
:1052EF003531353231353531353631363231363576
:1052FF003137323137343230353231323231343274
:10530F00323332323532323632343332343432345D
:10531F003532343632353132353232353532363147
:10532F00323633323635323636323731323734332E
:10533F003036333131333135333235333331333333
:10534F003233343333343633353133353633363411
:10535F00333635333731343131343132343133340C
:10536F0032333433313433323434353434363435F4
:10537F0032343534343535343632343634343635D8
:10538F0034363635303335303635313635323335D0
:10539F0032363533323534363536353630363631BA
:1053AF0032363234363237363331363332363534AD
:1053BF003636323636343730333731323732333799
:1053CF00333137333237333437343337353441426F
:1053DF00434445464748494A4B4C4D4E4F50515216
:1053EF00535455565758595A6162636465666768D6
:1053FF00696A6B6C6D6E6F70717273747576777896
:10540F00797A30313233343536373839607E21404E
:10541F002324255E262A28295F2D2B3D7B7D5B5D6E
:10542F007C3A3B3C3E2C2E3F2F202020202020205A
:10543F00202020202020474C4F42414C202020206C
:10544F00202020435443535320434F4445202020D2
:10545F002020202044435320434F44452020202028
:10546F0020204C5452205245504541544552202043
:10547F0020205350454544204449414C494E472034
:10548F00202053504545442043414C4C494E472022
:10549F00202020505443204E554D4245522020206D
:1054AF00202020564F494345204D455353414745F2
:1054BF00532020564F49434520504C4159424143B8
:1054CF004B202020494E56414C49442054595045B9
:1054DF00202020204F5554204F462052414E474503
:1054EF00202020494C4C4547414C2056414C5545B6
:1054FF0020204D5553542046494C4C204649454C8D
:10550F0044202020494C4C4547414C20434F4445B3
:10551F0020202044415441204143434550544544A9
:10552F0020204C494E45204E554D4245523A2020A1
:10553F002020555345522050524F4752414D4D490F
:10554F004E47555345522049443A202020202020D1
:10555F002020564F494345205245434F5244494E10
:10556F00472020494C4C4547414C20454E545259F9
:10557F00202020494C4C4547414C2047414E472065
:10558F002020202020434F4D504C4554454420208F
:10559F00202020474C4F42414C20454550524F4D03
:1055AF0020202020435443535320454550524F4D04
:1055BF00202020202044435320454550524F4D205A
:1055CF0020202020204C545220454550524F4D2032
:1055DF002020204449414C494E4720454550524FC9
:1055EF004D202043414C4C494E4720454550524F8A
:1055FF004D2020202050544320454550524F4D20E0
:10560F002020205245504541544552204545505287
:10561F004F4D2020494E495449414C495A494E4714
:10562F002020202052455045415445523A202020F9
:10563F00202020202020202020202020202020205B
:10564F00202020202020202020202020202020204B
:10565F00202020202020202020202020202020203B
:10566F00202020202020202020202020202020202B
:10567F00202020435443535320434F444520474158
:10568F004E472044435320434F44452047414E4704
:10569F0020202020525054522049442047414E4749
:1056AF002020202020525054522047414E47202086
:1056BF002020204449414C494E472047414E472026
:1056CF0020202043414C4C494E472047414E472014
:1056DF002020202020205054432047414E47202097
:0256EF00202079
:10E56E00BF31037FAA22BF32037FA322BF33037FB3
:10E57E00C122BF34037FC222BF35037FC322BF3601
:10E58E00037FC422BF37037FD722BF38037FAB225E
:0DE59E00BF39037FA822BF30037FA92222CE
:10E778009000E87464F0E4900000F030210B302041
:10E788002412E62312742880F530220B302016124A
:10E79800E65D12742880F530230B302008127F9331
:06E7A80012742880F52226
:107428009000E8E07012900000E0D394004009C298
:1074380021C222C223C22022900000E012AB8F7525
:107448004700754A01754D0275500375530475550B
:1074580005755706755907755C08755F0A75620BDF
:1074680075650F756810756B14756E1575711975DE
:10747800741A75771B757A1E757D1F758023758341
:1074880024758628758929758C2D758F2E75922FF0
:10749800759530759832759B33759D3475A0357523
:1074A800A33775A63875A96475AC6575AF6675B2EE
:1074B8006775B56E75B76F75B97075FD7175BB7801
:1074C80075BD7975BF7A75FD7B75C18275C3837586
:1074D800C58475C78575CA8C75CD8D75D08E75D2E6
:1074E8008F75D59675D89775DA9875DC9975DFA07C
:1074F80075E2A175E5A275E7A375EAAA75EDAB7506
:10750800F0AC75F2AD75F5B475F8B575FBB675FDEB
:10751800B775FFBE7602BF7605C07608C175FDC295
:10752800760EF07611F17614F27617FA761AFB7663
:107538001DFC7620FD7623FE7626FF0000762902C4
:10754800EFA502EDC702E26002ECAA800480028087
:107558000002DF0A0287A102E7080292F602D12B95
:1075680002944402D19E02959202E4B402BE2B0218
:107578009D6602D51B0296E002D58802982E02D697
:107588006202997C02EA9D02E69702DF9D12DEBF45
:1075980002DB81800002D3D102E2E802D283029AA0
:1075A800CA02DD3702E2A402E7AE028EEA80488012
:1075B80014804D80428023804780078008804102E4
:1075C80091A102BB4E02CEDA803602904B02CCEA81
:1075D8008008802C029C1802BD7B02D362802102A5
:1075E800892402CF5302D80B801602025702CFCA51
:1075F80002D874800B800C02D04102DD8802C6DFFD
:1076080002E5E8029FFB02ECD102D6CE02EFC702E8
:10761800DACA02F23702F23802F23902CD6702F210
:077628003AE4900000F0229B
:10EFA500E4900002F09000E87464F0900000E00442
:02EFB500F02248
:10EDC700126A2D126A3C7BFF7A55794112E9527F0C
:0FEDD70011126A13C227C224900000E004F02238
:10E26000302440900001E0FFC224BF2A0790000044
:10E27000E004F022EF6423702A7F231269E4900007
:10E2800002E004F0E0C394034013C221C222C2237F
:10E29000C220E4900000F012E21B026A4B900000E2
:03E2A0007402F015
:01E2A3002258
:10ECAA007BFF7A55794112E952126A3C7F11126A46
:10ECBA001312F011E490003DF07F2A1269E4C22792
:07ECCA00900000E004F022BD
:10DF0A00302446900001E0F568C224E568642A607E
:10DF1A0038AF6812EFE65022AF681269E490003D0C
:10DF2A00E02403F582E43400F583E568F090003DCF
:10DF3A00E004F0900000E004F0227BFF7A5579714A
:09DF4A0012E95290000074FAF093
:01DF530022AB
:1087A100202403028923900001E0FFC224BF2A078D
:1087B1009000007403F022EF642360030289141215
:1087C10069E4900004E06439707CA3E06439707658
:1087D100A3E064397070D228900003E0FFB431083F
:1087E100E4900036F0028870EFB43208E49000376C
:1087F100F0028883EFB433028043900003E0FFB4BA
:108801003408E4900038F00288B1EFB43508E49000
:108811000039F00288C2EFB43608E490003BF00260
:1088210088D8EFB437028015900003E0FFB438090F
:108831009000357401F002890DEFB4390B7BFF7A9A
:1088410055798102891AC228900003E0FFB43016DD
:10885100A3E0B43011A3E0B4300CA3E0B43007902E
:108861000000740AF022EFB4310C12DA6D50079057
:108871000000740FF022900003E0B4320C12DA0D04
:1088810050079000007414F022900003E0B43311FB
:10889100A3E0B4300C12EDA650079000007419F05B
:1088A10022900003E0B4340FA3E0B4300A12EF1CAD
:1088B100900000741EF022900003E0B4350A12ED1E
:1088C100409000007423F022900003E0B4360FA31F
:1088D100E0B4300A12EF319000007428F0229000C9
:1088E10003E0FFB43716A3E0B43011A3E0B4300CB9
:1088F100A3E0B43007900000742DF022EFB43813D8
:10890100900004E0B4300C12EDA650079000007402
:1089110037F0227BFF7A55797112E9529000007489
:02892100FAF06A
:018923002231
:10E7080090003C740BF090003D7407F0E490004AD0
:10E71800F0A3F090004C7481F0E490004DF0A3F069
:10E728007BFF7A54794112E95212E97D7F1E126A01
:08E73800139000007432F0227E
:1092F60012D0B6D3900075E09466900074E09400A6
:10930600400A12E94C90000074FAF022900074E0D2
:10931600FEA3E0FF904C6F75F00912AB83EE75F07B
:1093260009A42583F583E493900041F0904C707571
:10933600F009EF12AB83EE75F009A42583F583E4FB
:1093460093900042F0900074A3E0904C7175F00980
:1093560012AB83EE75F009A42583F583E4939000A0
:1093660043F0904C7275F009EF12AB83EE75F0097D
:10937600A42583F583E493900044F0900074A3E061
:10938600904C7375F00912AB83EE75F009A4258332
:10939600F583E493FD900045F0904C7475F009EF69
:1093A60012AB83EE75F009A42583F583E493900050
:1093B60046F0900074A3E0904C7575F00912AB83EB
:1093C600EE75F009A42583F583E493900047F090A9
:1093D6004C7675F009EF12AB83EE75F009A4258380
:1093E600F583E493900048F0900074A3E0904C77E6
:1093F60075F00912AB83EE75F009A42583F583E4B5
:1094060093900049F0ED6015900045E075F010A4CA
:10941600243FF9744435F0FA7BFF12E95290004676
:10942600E0FF601175F010A4243FF9744435F0FA9A
:0E9436007BFF12E983900041E0900000F022DD
:10D12B0090003C7410F090003D7407F090004AE4BE
:10D13B00F0A37481F0E490004CF030281490004D73
:10D14B00F0A3F07BFF7A56798112E95212E97D80C8
:10D15B0036900036E0FF90004DE4F0A3EFF07BFF3C
:10D16B007A54795112E95212E97D7F0D126A1390AC
:10D17B000004E0FF1269E4900005E0FF1269E490FF
:10D18B000006E0FF1269E47F1E126A139000007420
:03D19B0032F0224D
:1094440012D0B6D3900075E09400900074E09400BC
:10945400400A12E94C90000074FAF022900074E083
:10946400FEA3E0FF90501E75F00912AB83EE75F079
:1094740009A42583F583E493900041F090501F756F
:10948400F009EF12AB83EE75F009A42583F583E4AC
:1094940093900042F0900074A3E090502075F0097E
:1094A40012AB83EE75F009A42583F583E493900051
:1094B40043F090502175F009EF12AB83EE75F0097B
:1094C400A42583F583E493900044F0900074A3E012
:1094D40090502275F00912AB83EE75F009A4258330
:1094E400F583E493FD900045F090502375F009EF67
:1094F40012AB83EE75F009A42583F583E493900001
:1095040046F0900074A3E090502475F00912AB83E8
:10951400EE75F009A42583F583E493900047F09059
:10952400502575F009EF12AB83EE75F009A425837D
:10953400F583E493900048F0900074A3E0905026E3
:1095440075F00912AB83EE75F009A42583F583E465
:1095540093900049F0ED6015900045E075F010A47B
:10956400240EF9745035F0FA7BFF12E9529000464C
:10957400E0FF601175F010A4240EF9745035F0FA70
:0E9584007BFF12E983900041E0900000F0228E
:10D19E0090003C7415F090003D7407F090004AE446
:10D1AE00F0A37481F0E490004CF030281490004D00
:10D1BE00F0A3F07BFF7A56799112E95212E97D8045
:10D1CE0036900037E0FF90004DE4F0A3EFF07BFFC8
:10D1DE007A54796112E95212E97D7F0C126A13902A
:10D1EE000004E0FF1269E4900005E0FF1269E4908C
:10D1FE000006E0FF1269E47F1E126A1390000074AD
:03D20E0032F022D9
:1095920012D0B6D3900075E09400900074E094006D
:1095A200400A12E94C90000074FAF022900074E034
:1095B200FEA3E0FF90503775F00912AB83EE75F011
:1095C20009A42583F583E493900041F09050387507
:1095D200F009EF12AB83EE75F009A42583F583E45D
:1095E20093900042F0900074A3E090503975F00916
:1095F20012AB83EE75F009A42583F583E493900002
:1096020043F090503A75F009EF12AB83EE75F00912
:10961200A42583F583E493900044F0900074A3E0C2
:1096220090503B75F00912AB83EE75F009A42583C7
:10963200F583E493FD900045F090503C75F009EFFE
:1096420012AB83EE75F009A42583F583E4939000B1
:1096520046F0900074A3E090503D75F00912AB8380
:10966200EE75F009A42583F583E493900047F0900A
:10967200503E75F009EF12AB83EE75F009A4258315
:10968200F583E493900048F0900074A3E090503F7B
:1096920075F00912AB83EE75F009A42583F583E416
:1096A20093900049F0ED6015900045E075F010A42C
:1096B2002427F9745035F0FA7BFF12E952900046E4
:1096C200E0FF601175F010A42427F9745035F0FA08
:0E96D2007BFF12E983900041E0900000F0223F
:10E4B4007BFF7A54797112E9527BFF7A55795112B4
:10E4C400E9837F0E126A13900005E0FF1269E4905D
:10E4D4000006E0FF1269E47F1A126A1390003C748C
:0FE4E4001AF090003D7404F09000007432F022A2
:10BE2B003029079000007403F022900007E064397A
:10BE3B007041A3E06439703BA3E064397035900026
:10BE4B003C741BF090003D7407F07BFF7A5679A190
:10BE5B0012E952D22890004AE4F0A37481F0E490E6
:10BE6B00004CF090004DF0A3F012E97D7F1E126A9A
:10BE7B0013804B12E97D7F1E126A1312D945900075
:10BE8B0076E0FEA3E0FFD39400EE94004037EF94EE
:10BE9B00FBEE9400502F90003C741BF090003D740F
:10BEAB0007F090004AE4F0A37481F0E490004CF0AA
:10BEBB00EF24FFFFEE34FF90004DF0A3EFF0900066
:0FBECB00007432F02212E94C90000074FAF02259
:109D6600D3900075E094FF900074E094FF400A12CF
:109D7600E94C90000074FAF022900074E0FEA3E033
:109D8600FF90505075F00912AB83EE75F009A425CB
:109D960083F583E493900041F090505175F009EFFC
:109DA60012AB83EE75F009A42583F583E493900046
:109DB60042F0900074A3E090505275F00912AB8304
:109DC600EE75F009A42583F583E493900043F090A3
:109DD600505375F009EF12AB83EE75F009A4258395
:109DE600F583E493900044F0900074A3E0905054FF
:109DF60075F00912AB83EE75F009A42583F583E4AB
:109E060093FD900045F090505575F009EF12AB8325
:109E1600EE75F009A42583F583E493900046F0904F
:109E26000074A3E090505675F00912AB83EE75F0FE
:109E360009A42583F583E493900047F09050577565
:109E4600F009EF12AB83EE75F009A42583F583E4E0
:109E560093900048F0900074A3E090505875F00974
:109E660012AB83EE75F009A42583F583E493900085
:109E760049F0ED6015900045E075F010A42440F916
:109E8600745035F0FA7BFF12E952900046E0FF600D
:109E96001175F010A42440F9745035F0FA7BFF12C6
:0B9EA600E983900041E0900000F022F2
:10D51B0090003C741FF090003D7407F090004AE4BB
:10D52B00F0A37481F090004C7410F0302815E49047
:10D53B00004DF0A3F07BFF7A5679C112E95212E944
:10D54B007D802E900038E0FF90004DE4F0A3EFF0CB
:10D55B007BFF7A54798112E95212E97D7F0F126AAF
:10D56B0013900005E0FF1269E4900006E0FF1269DA
:0DD57B00E47F1E126A139000007432F0224B
:1096E00012D0B6D3900075E09400900074E094001E
:1096F000400A12E94C90000074FAF022900074E0E5
:10970000FEA3E0FF90508975F00912AB83EE75F06F
:1097100009A42583F583E493900041F090508A7565
:10972000F009EF12AB83EE75F009A42583F583E40D
:1097300093900042F0900074A3E090508B75F00974
:1097400012AB83EE75F009A42583F583E4939000B2
:1097500043F090508C75F009EF12AB83EE75F00971
:10976000A42583F583E493900044F0900074A3E073
:1097700090508D75F00912AB83EE75F009A4258326
:10978000F583E493FD900045F090508E75F009EF5D
:1097900012AB83EE75F009A42583F583E493900062
:1097A00046F0900074A3E090508F75F00912AB83DF
:1097B000EE75F009A42583F583E493900047F090BB
:1097C000509075F009EF12AB83EE75F009A4258374
:1097D000F583E493900048F0900074A3E0905091DA
:1097E00075F00912AB83EE75F009A42583F583E4C7
:1097F00093900049F0ED6015900045E075F010A4DD
:109800002459F9745035F0FA7BFF12E95290004662
:10981000E0FF601175F010A42459F9745035F0FA86
:0E9820007BFF12E983900041E0900000F022EF
:10D5880090003C7424F090003D7407F090004A1419
:10D59800F0A374C1F090004C7410F0302815E4909A
:10D5A800004DF0A3F07BFF7A5679D112E95212E9C7
:10D5B8007D802E900039E0FF90004DE4F0A3EFF05D
:10D5C8007BFF7A54799112E95212E97D7F0F126A32
:10D5D80013900005E0FF1269E4900006E0FF12696D
:0DD5E800E47F1E126A139000007432F022DE
:10982E0012D0B6D3900075E09400900074E09400CE
:10983E00400A12E94C90000074FAF022900074E095
:10984E00FEA3E0FF9050C275F00912AB83EE75F0E7
:10985E0009A42583F583E493900041F09050C375DD
:10986E00F009EF12AB83EE75F009A42583F583E4BE
:10987E0093900042F0900074A3E09050C475F009EC
:10988E0012AB83EE75F009A42583F583E493900063
:10989E0043F09050C575F009EF12AB83EE75F009E9
:1098AE00A42583F583E493900044F0900074A3E024
:1098BE009050C675F00912AB83EE75F009A425839E
:1098CE00F583E493FD900045F09050C775F009EFD5
:1098DE0012AB83EE75F009A42583F583E493900013
:1098EE0046F0900074A3E09050C875F00912AB8357
:1098FE00EE75F009A42583F583E493900047F0906C
:10990E0050C975F009EF12AB83EE75F009A42583EB
:10991E00F583E493900048F0900074A3E09050CA51
:10992E0075F00912AB83EE75F009A42583F583E477
:10993E0093900049F0ED6015900045E075F010A48D
:10994E002492F9745035F0FA7BFF12E952900046DA
:10995E00E0FF601175F010A42492F9745035F0FAFE
:0E996E007BFF12E983900041E0900000F022A0
:10D6620090003C7429F090003D7407F090004A74D9
:10D672000DF0A37401F0E490004CF03028149000F7
:10D682004DF0A3F07BFF7A5679E112E95212E97D5F
:10D69200802E90003BE0FF90004DE4F0A3EFF07B82
:10D6A200FF7A5479A112E95212E97D7F0D126A13B1
:10D6B200900005E0FF1269E4900006E0FF1269E4C1
:0CD6C2007F1E126A139000007432F022E8
:10997C0012D0B6D3900075E094FF900074E094FF81
:10998C00400A12E94C90000074FAF022900074E046
:10999C00FEA3E0FF9050DB75F00912AB83EE75F07F
:1099AC0009A42583F583E493900041F09050DC7575
:1099BC00F009EF12AB83EE75F009A42583F583E46F
:1099CC0093900042F0900074A3E09050DD75F00984
:1099DC0012AB83EE75F009A42583F583E493900014
:1099EC0043F09050DE75F009EF12AB83EE75F00981
:1099FC00A42583F583E493900044F0900074A3E0D5
:109A0C009050DF75F00912AB83EE75F009A4258335
:109A1C00F583E493FD900045F09050E075F009EF6C
:109A2C0012AB83EE75F009A42583F583E4939000C3
:109A3C0046F0900074A3E09050E175F00912AB83EE
:109A4C00EE75F009A42583F583E493900047F0901C
:109A5C0050E275F009EF12AB83EE75F009A4258383
:109A6C00F583E493900048F0900074A3E09050E3E9
:109A7C0075F00912AB83EE75F009A42583F583E428
:109A8C0093900049F0ED6015900045E075F010A43E
:109A9C0024CBF9745035F0FA7BFF12E95290004652
:109AAC00E0FF601175F010A424CBF9745035F0FA76
:0E9ABC007BFF12E983900041E0900000F02251
:10EA9D003023079000007401F02290003C742EF09A
:10EAAD0090003D7407F07BFF7A5479B112E9521250
:0EEABD00E97D7F1E126A139000007432F02271
:10E69700302907900000742FF02290000AE06438B8
:10E6A7006005A3E0B4390A12E94C90000074FAF04F
:10E6B700227BFF7A55796112E95290000AE0540FE4
:09E6C700F5509000007430F022BF
:10DF9D0090000AE064386005A3E0B4390A12E94C38
:10DFAD0090000074FAF0227BFF7A5479C112E95285
:10DFBD0090000AE0540FF550D202D20A900121E0F0
:10DFCD00F5281282E37BFF7A55799112E952C2024C
:09DFDD00C20A90000074FEF0225B
:10DEBF0090000AE0540FF550302102D2001282F583
:10DECF0030211B201304E54170F91282ECC2007B54
:10DEDF00FF7A55799112E95290000074FEF03022CA
:10DEEF0019201104E54170F91282EC7BFF7A557904
:0BDEFF009112E95290000074FEF02226
:10DB8100302456900001E0FF900034F0C224126965
:10DB9100E4900034E0FF12EFE65021900034E0FF02
:10DBA10090003DE02403F582E43400F583EFF0902A
:10DBB100003DE004F0900000E004F022900034E029
:10DBC100B42A079000007403F0227BFF7A55797123
:0ADBD10012E95290000074FAF022ED
:10D3D10030246A900001E0FF900034F0C224126909
:10D3E100E4900034E0FFB42A0B90003CE090000090
:10D3F100F0D22922EFB4230B90003CE0900000F022
:10D40100C22922900034E0FF12EFE650219000344F
:10D41100E0FF90003DE02403F582E43400F583EF62
:10D42100F090003DE004F0900000E004F0227BFF6A
:0ED431007A55797112E95290000074FAF022D7
:10E2E80030243F900001E0FF900034F01269E4C24E
:10E2F80024900034E0FFB42A0B90003CE09000002A
:10E30800F0D22922EFB4230B90003CE0900000F0FB
:10E31800C229227BFF7A55797112E9529000007464
:03E32800FAF022E6
:10D2830090003C7438F090003D7407F090004A74AD
:10D293000DF0A37401F0E490004CF03028149000DA
:10D2A3004DF0A3F07BFF7A5679B112E95212E97D72
:10D2B3008032900035E024FFFEE434FF90004DF00F
:10D2C300A3CEF07BFF7A56793112E95212E97D7FC2
:10D2D3000C126A13900005E0FF1269E4900006E067
:10D2E300FF1269E47F1E126A139000007432F02269
:109ACA0012D0B6D3900075E094FF900074E094FF32
:109ADA00400A12E94C90000074FAF022900074E0F7
:109AEA00FEA3E0FF90514575F00912AB83EE75F0C5
:109AFA0009A42583F583E493900041F090514675BB
:109B0A00F009EF12AB83EE75F009A42583F583E41F
:109B1A0093900042F0900074A3E090514775F009C9
:109B2A0012AB83EE75F009A42583F583E4939000C4
:109B3A0043F090514875F009EF12AB83EE75F009C6
:109B4A00A42583F583E493900044F0900074A3E085
:109B5A0090514975F00912AB83EE75F009A425837B
:109B6A00F583E493FD900045F090514A75F009EFB2
:109B7A0012AB83EE75F009A42583F583E493900074
:109B8A0046F0900074A3E090514B75F00912AB8334
:109B9A00EE75F009A42583F583E493900047F090CD
:109BAA00514C75F009EF12AB83EE75F009A42583C9
:109BBA00F583E493900048F0900074A3E090514D2F
:109BCA0075F00912AB83EE75F009A42583F583E4D9
:109BDA0093900049F0ED6015900045E075F010A4EF
:109BEA002435F9745135F0FA7BFF12E95290004698
:109BFA00E0FF601175F010A42435F9745135F0FABC
:0E9C0A007BFF12E983900041E0900000F02201
:0ADD3700900044E0FF70033029382B
:10DD4100126A1312EC0212C98F8F68900042E052DE
:10DD510068E56860047F3180027F301269E4302910
:10DD610017C229E5682430900023F0900033740134
:08DD7100F090000074F0F022B4
:0FDD7900900047E0FF126A13900000E004F022D0
:10E2A400302440900001E0FF900034F0C224126951
:10E2B400E4900034E0FFB42A079000007403F022D5
:10E2C40012EFE6500F900034E090000DF090000043
:10E2D400E004F0227BFF7A55797112E95290000034
:04E2E40074FAF022B6
:10E7AE00302432900001E0FF900034F0C224BF2AE2
:10E7BE00079000007403F022900034E0B423079019
:10E7CE000000E004F0227BFF7A55797112E9529035
:06E7DE00000074FAF022B5
:108EEA00302879900003E06438707190004DF0A347
:108EFA00F012EC02900078EEF0A3EFF012C98F8F17
:108F0A005C90003E7401F090000DE0B431139000C3
:108F1A0042E0425C900078E0FEA3E0FFAD5C12C93B
:108F2A004E90000DE0B43014900042E0F4525C9090
:108F3A000078E0FEA3E0FFAD5C12C94E90004EE05F
:108F4A0004F0700690004DE004F0C390004EE094E7
:108F5A001490004DE09400409802903B302878909D
:108F6A000003E06433707090004DF0A3F012EC023D
:108F7A00900078EEF0A3EFF012C98F8F5C90003E5C
:108F8A007401F090000DE0B43113900042E0425CAD
:108F9A00900078E0FEA3E0FFAD5C12C94E90000D90
:108FAA00E0B43014900042E0F4525C900078E0FEA5
:108FBA00A3E0FFAD5C12C94E90004EE004F07006CB
:108FCA0090004DE004F0C390004EE094FA90004DFA
:108FDA00E094004098805312EC02900078EEF0A3DF
:108FEA00EFF012C98F8F5C90003E7401F090000D73
:108FFA00E0B43118900042E0425C900078E0FEA3B1
:10900A00E0FFAD5C12C94E12EF46801E90000DE0E3
:10901A00B4301E900042E0F4525C900078E0FEA367
:10902A00E0FFAD5C12C94E12EF4690000074FEF0EC
:10903A00227BFF7A55797112E95290000074FAF096
:01904A002203
:10D04100900044E0FF7003302956126A1312EC027B
:10D05100900078EEF0A3EFF0E4F55C900042E0FF81
:10D06100E55CC39F5027900078E475F00112AB6D29
:10D07100AFF0FE12C98F8F5D7423255CF582E43415
:10D0810000F583E55DF01269E4055C80CE3029107E
:10D09100C229E55C04900033F090000074F0F022A6
:10D0A10090003D740AF0900047E0FF126A1390006F
:05D0B10000E004F02284
:10CEDA00302475900001E0FF900034F0C2241269FA
:10CEEA00E4900034E0FFB42A079000007403F022B3
:10CEFA00EFB42308900000E004F0803912EFE65006
:10CF0A0038900034E0FF90003DE0FE04F074032EF8
:10CF1A00F582E43400F583EFF0900042E02409FF43
:10CF2A00E433FE90003DE0D39FEE6480F87480986D
:10CF3A004016900000E004F0227BFF7A55797112C6
:09CF4A00E95290000074FAF02293
:10E5E800302437900001E0FF900034F0C224126913
:10E5F800E4900034E0FFB42A079000007403F0228E
:10E60800EFB42307900000E004F0227BFF7A5579ED
:0BE618007112E95290000074FAF02229
:109FFB00302874900003E06434706C90004DF0A333
:10A00B00F012EC02900078EEF0A3EFF090003D74AC
:10A01B000AF0E4F55C900042E0FFE55CC39F50273B
:10A02B00900078E475F00112AB6DAFF0FE90003D3F
:10A03B00E0FD04F074032DF582E43400F583E0FDBC
:10A04B0012C94E055C80CE90004EE004F070069075
:10A05B00004DE004F0C390004EE0946490004DE09E
:10A06B009400409D02A12E302873900003E06436CB
:10A07B00706B90004DF0A3F012EC02900078EEF0B4
:10A08B00A3EFF090003D740AF0E4F55C900042E021
:10A09B00FFE55CC39F5027900078E475F00112AB8D
:10A0AB006DAFF0FE90003DE0FD04F074032DF582E2
:10A0BB00E43400F583E0FD12C94E055C80CE9000C0
:10A0CB004EE004F0700690004DE004F0C390004E9B
:10A0DB00E0946490004DE09400409D804612EC02A9
:10A0EB00900078EEF0A3EFF090003D740AF0E4F5E9
:10A0FB005C900042E0FFE55CC39F5027900078E442
:10A10B0075F00112AB6DAFF0FE90003DE0FD04F079
:10A11B0074032DF582E43400F583E0FD12C94E057E
:10A12B005C80CE7BFF7A55799112E95290000074D6
:03A13B00FEF02211
:10D3620030246B900001E0FF900034F0C224126977
:10D37200E4900034E0FFB42A079000007403F02226
:10D3820012EFE6501A900034E0FF90003DE0FE04F8
:10D39200F074032EF582E43400F583EFF080107B05
:10D3A200FF7A55797112E95290000074FAF02290D6
:10D3B2000042E02409FFE433FE90003DE0D39FEEFB
:0FD3C2006480F87480984006900000E004F02228
:10BB4E00900044E0FF700620290302BBF9126A132D
:10BB5E0012EC02900078EEF0A3EFF012C98F127281
:10BB6E00B5900042E0B40110900071E0FF1269E45C
:10BB7E00900071E0900023F0900042E0B40220901B
:10BB8E000070E0FF1269E4900071E0FF1269E4902A
:10BB9E000070E0900023F0900071E0900024F0908F
:10BBAE000042E06403703090006FE0FF1269E49091
:10BBBE000070E0FF1269E4900071E0FF1269E490FA
:10BBCE00006FE0900023F0900070E0900024F09061
:10BBDE000071E0900025F0302911C229900042E05A
:10BBEE00900033F090000074F0F022900047E0FFD8
:10BBFE00126A1390003D740AF0900000E004F022E7
:1091A10012730B50030292EC1272E38F5C90004831
:1091B100E0FFE55CC39F50030292EC900049E0FFA1
:1091C100E55CD39F40030292EC30283E900003E01F
:1091D1006431703690004DF0A3F012EC02900078EB
:1091E100EEF0A3EFF0AD5C12C94E90004EE004F03A
:1091F100700690004DE004F0C390004EE09433906F
:10920100004DE0940040D30292DC30283E900003F0
:10921100E06432703690004DF0A3F012EC02900041
:1092210078EEF0A3EFF0AD5C12C94E90004EE00471
:10923100F0700690004DE004F0C390004EE0947091
:1092410090004DE0940040D30292DC30283D900024
:1092510003E06433703590004DF0A3F012EC0290FE
:109261000078EEF0A3EFF0AD5C12C94E90004EE035
:1092710004F0700690004DE004F0C390004EE094BD
:10928100FA90004DE0940040D3805030283D90008A
:1092910003E06438703590004DF0A3F012EC0290B9
:1092A1000078EEF0A3EFF0AD5C12C94E90004EE0F5
:1092B10004F0700690004DE004F0C390004EE0947D
:1092C1001490004DE0940040D3801012EC02900005
:1092D10078EEF0A3EFF0AD5C12C94E7BFF7A5579C1
:1092E1009112E95290000074FEF02212E94C9000B4
:0592F1000074FAF022F8
:10904B0012730B50030291971272E38F5C900048DE
:10905B00E0FFE55CC39F400B900049E0FFE55CD36C
:10906B009F4007E55C600302919730283E90000318
:10907B00E06431703690004DF0A3F012EC029000DA
:10908B0078EEF0A3EFF0AD5C12C94E90004EE00409
:10909B00F0700690004DE004F0C390004EE0943366
:1090AB0090004DE0940040D302918730283E900011
:1090BB0003E06432703690004DF0A3F012EC029096
:1090CB000078EEF0A3EFF0AD5C12C94E90004EE0CD
:1090DB0004F0700690004DE004F0C390004EE09455
:1090EB007090004DE0940040D302918730283D9062
:1090FB000003E06433703590004DF0A3F012EC02E6
:10910B00900078EEF0A3EFF0AD5C12C94E90004EDC
:10911B00E004F0700690004DE004F0C390004EE0C8
:10912B0094FA90004DE0940040D3805030283D904D
:10913B000003E06438703590004DF0A3F012EC02A0
:10914B00900078EEF0A3EFF0AD5C12C94E90004E9C
:10915B00E004F0700690004DE004F0C390004EE088
:10916B00941490004DE0940040D3801012EC0290C8
:10917B000078EEF0A3EFF0AD5C12C94E7BFF7A5591
:10918B00799112E95290000074FEF02212E94C9092
:06919B00000074FAF0224E
:10CCEA00900044E0FF700330295E126A1312EC02CE
:10CCFA00900078EEF0A3EFF012C98F8F5C12CA6130
:10CD0A00E4F55C746F255CF582E43400F583E0FF9A
:10CD1A007423255CF582E43400F583EFF0746F2503
:10CD2A005CF582E43400F583E0FF1269E4055CE512
:10CD3A005CC3940440CD30290FC229900033740398
:10CD4A00F090000074F0F022900047E0FF126A139E
:0DCD5A0090003D740AF0900000E004F0220B
:109C18007F0A12ACB08F5CE55C7003029D4430286B
:109C280040900003E06431703890004DF0A3F012CA
:109C3800EC02900078EEF0A3EFF0E55C14FD12C999
:109C48004E90004EE004F0700690004DE004F0C322
:109C580090004EE0943390004DE0940040D1029D76
:109C68002E302840900003E06432703890004DF0A8
:109C7800A3F012EC02900078EEF0A3EFF0E55C148C
:109C8800FD12C94E90004EE004F0700690004DE0C1
:109C980004F0C390004EE0947090004DE0940040B2
:109CA800D1029D2E30283F900003E0643370379036
:109CB800004DF0A3F012EC02900078EEF0A3EFF064
:109CC800E55C14FD12C94E90004EE004F070069059
:109CD800004DE004F0C390004EE094FA90004DE08F
:109CE800940040D18040302841900003E0643870EF
:109CF8003990004DF0A3F012EC02900078EEF0A33A
:109D0800EFF0E55C14FD12C94E90004EE004F070CF
:109D18000690004DE004F0C390004EE094149000CB
:109D28004DE0940040D17BFF801812EC029000783F
:109D3800EEF0A3EFF0E55C14FD12C94EE55C7BFF85
:109D4800600E7A55799112E95290000074FEF02263
:0E9D58007A55791112E95290000074FAF02247
:10BD7B00900044E0FF700620290302BE16126A13DE
:10BD8B0012EC02900078EEF0A3EFF012C98F127252
:10BD9B00B5900078E475F00112AB6DAFF0FE12C9EF
:10BDAB008F127299900070E0FF900023F0A3F012B5
:10BDBB0069E4900071E0FF1269E4900078E475F09B
:10BDCB000112AB6DAFF0FE12C98F12729990006F1A
:10BDDB00E0FF900025F0900070E0900026F09000BE
:10BDEB0071E0900027F01269E4900070E0FF126997
:10BDFB00E4900071E0FF1269E430290FC229900032
:10BE0B00337405F090000074F0F022900047E0FFCF
:10BE1B00126A1390003D740AF0900000E004F022C7
:1089240090000DE0540F75F00AA4FFA3E0540F2F3C
:10893400F55C900010E0540F75F00AA4FDACF090C3
:10894400000FE0540F75F064A42DFFE5F03CFE9099
:108954000011E0540F7C002FF55FEC3EF55EE55C02
:10896400C39401401DE55CD394145016C3E55F9491
:1089740001E55E9400400BD3E55F94FAE55E940054
:10898400400A12E94C90000074FAF0223028589002
:108994000003E06431705090004DF0A3F012EC023B
:1089A400900078EEF0A3EFF0900078E475F00112F7
:1089B400AB6DAFF0FEAD5C12C94E900078E0FEA343
:1089C400E0FFAD5F12C94E90004EE004F0700690D7
:1089D400004DE004F0C390004EE0943390004DE06D
:1089E400940040B9028A8F302857900003E0643223
:1089F400704F90004DF0A3F012EC02900078EEF06E
:108A0400A3EFF0900078E475F00112AB6DAFF0FEC7
:108A1400AD5C12C94E900078E0FEA3E0FFAD5F129A
:108A2400C94E90004EE004F0700690004DE004F052
:108A3400C390004EE0947090004DE0940040B980E3
:108A44004A12EC02900078EEF0A3EFF0900078E484
:108A540075F00112AB6DAFF0FEAD5C12C94E900023
:108A640010E0540F75F00AA4FF90000FE0540F7546
:108A7400F064A42FFF900011E0540F2FF55C9000D8
:108A840078E0FEA3E0FFAD5C12C94E7BFF7A557916
:0B8A94009112E95290000074FEF022E5
:10CF5300900044E0FF7003302956126A1312EC026A
:10CF6300900078EEF0A3EFF0E4F55C900042E0FF70
:10CF7300E55CC39F5027900078E475F00112AB6D18
:10CF8300AFF0FE12C98F8F5D7423255CF582E43404
:10CF930000F583E55DF01269E4055C80CE3029106D
:10CFA300C229E55C04900033F090000074F0F02295
:10CFB300900047E0FF126A1390003D740AF0D227F5
:07CFC300900000E004F022E1
:10D80B00302465900001E0FF900034F0C224BF2A61
:10D81B00079000007403F022900034E0FFB423085B
:10D82B00900000E004F0803DEF547FFF1269E4901C
:10D83B000034E0547FFF90003DE0FE04F074032EB3
:10D84B00F582E43400F583EFF0900042E02409FF09
:10D85B00E433FE90003DE0D39FEE6480F874809833
:09D86B004006900000E004F022E8
:1002570090000FE0FFC394304042EFD39433503CFB
:10026700A3E0C39430403590000FE0D39439502C6D
:10027700900011E0FFC394304022EFD39439501C13
:10028700A3E0FFC394304014EFD39439500EA3E09A
:10029700FFC394304006EFD394394003024435122C
:1002A700EC02900078EEF0A3EFF090003D740AF0B6
:1002B70090000DE0643060030203B2A3E064316094
:1002C700030203B2900017E0FF64306008EF643167
:1002D70060030203B2900018E0642060030203B2D7
:1002E7007F1012AD9EEFD3940050030203B27F102C
:1002F70012AD9EEFC3943540030203B230287490C9
:100307000003E06435706C90004DF0A3F012EC022E
:10031700900078EEF0A3EFF090003D740AF0E4F55A
:100327005C900042E0FFE55CC39F5027900078E4B3
:1003370075F00112AB6DAFF0FE90003DE0FD04F0EB
:1003470074032DF582E43400F583E0FD12C94E05F0
:100357005C80CE90004EE004F0700690004DE00403
:10036700F0C390004EE094E790004DE09403409D69
:10037700024425E4F55C900042E0FFE55CC39F5032
:1003870027900078E475F00112AB6DAFF0FE900096
:100397003DE0FD04F074032DF582E43400F583E0BD
:1003A700FD12C94E055C80CE02442590000DE06425
:1003B7003060030204ADA3E0643260030204AD9031
:1003C7000017E0FF64306008EF643160030204AD9A
:1003D700900018E0642060030204AD7F1012AD9E08
:1003E700EFD3943350030204AD7F1012AD9EEFC3D9
:1003F70094A540030204AD302874900003E06435EF
:10040700706C90004DF0A3F012EC02900078EEF0C3
:10041700A3EFF090003D740AF0E4F55C900042E031
:10042700FFE55CC39F5027900078E475F00112AB9D
:100437006DAFF0FE90003DE0FD04F074032DF582F2
:10044700E43400F583E0FD12C94E055C80CE9000D0
:100457004EE004F0700690004DE004F0C390004EAB
:10046700E094E790004DE09403409D024425E4F5B5
:100477005C900042E0FFE55CC39F5027900078E462
:1004870075F00112AB6DAFF0FE90003DE0FD04F09A
:1004970074032DF582E43400F583E0FD12C94E059F
:1004A7005C80CE02442590000DE0643060030205B5
:1004B7007BA3E06433600302057B90001CE06420AB
:1004C700600302057B302874900003E06435706C8C
:1004D70090004DF0A3F012EC02900078EEF0A3EF3D
:1004E700F090003D740AF0E4F55C900042E0FFE50F
:1004F7005CC39F5027900078E475F00112AB6DAF95
:10050700F0FE90003DE0FD04F074032DF582E43425
:1005170000F583E0FD12C94E055C80CE90004EE0E9
:1005270004F0700690004DE004F0C390004EE09494
:10053700E790004DE09403409D024425E4F55C906C
:100547000042E0FFE55CC39F5027900078E475F018
:100557000112AB6DAFF0FE90003DE0FD04F07403B7
:100567002DF582E43400F583E0FD12C94E055C8069
:10057700CE02442590000DE0643060030206A1A37B
:10058700E0643460030206A1900018E06420600371
:100597000206A1900014E0FFC3943050030206A1A5
:1005A700EFD3943740030206A1900016E0FFC394EF
:1005B7003050030206A1EFD3943740030206A190FF
:1005C7000015E0FFC3943050030206A1EFD394391E
:1005D70040030206A1900017E0FFC39430500302C6
:1005E70006A1EFD3943940030206A1302874900086
:1005F70003E06435706C90004DF0A3F012EC0290AC
:100607000078EEF0A3EFF090003D740AF0E4F55C9B
:10061700900042E0FFE55CC39F5027900078E475A7
:10062700F00112AB6DAFF0FE90003DE0FD04F074F9
:10063700032DF582E43400F583E0FD12C94E055C15
:1006470080CE90004EE004F0700690004DE004F07C
:10065700C390004EE094E790004DE09403409D0264
:100667004425E4F55C900042E0FFE55CC39F50271A
:10067700900078E475F00112AB6DAFF0FE90003D8D
:10068700E0FD04F074032DF582E43400F583E0FD0A
:1006970012C94E055C80CE02442590000DE06430FF
:1006A70060030207C7A3E0643560030207C7900031
:1006B70018E0642060030207C7900014E0FFC394AA
:1006C7003050030207C7EFD3943240030207C790A5
:1006D7000016E0FFC3943050030207C7EFD39432EC
:1006E70040030207C7900015E0FFC3943050030290
:1006F70007C7EFD3943940030207C7900017E0FFFD
:10070700C3943050030207C7EFD39439400302075D
:10071700C7302874900003E06435706C90004DF08A
:10072700A3F012EC02900078EEF0A3EFF090003DFA
:10073700740AF0E4F55C900042E0FFE55CC39F506B
:1007470027900078E475F00112AB6DAFF0FE9000D2
:100757003DE0FD04F074032DF582E43400F583E0F9
:10076700FD12C94E055C80CE90004EE004F0700685
:1007770090004DE004F0C390004EE094E790004DE8
:10078700E09403409D024425E4F55C900042E0FFBD
:10079700E55CC39F5027900078E475F00112AB6DBC
:1007A700AFF0FE90003DE0FD04F074032DF582E408
:1007B7003400F583E0FD12C94E055C80CE02442566
:1007C70090000DE064306003020945A3E0643660E1
:1007D7000302094590001CE064206003020945906C
:1007E7000014E0FFC394305003020945EFD394315E
:1007F7004003020945900016E0FFC39430500302FE
:100807000945EFD394314003020945900018E0FFF2
:10081700C394305003020945EFD3943140030209D2
:100827004590001AE0FFC394305003020945EFD307
:1008370094314003020945900015E0FFC3943050FE
:1008470003020945EFD39437400302094590001787
:10085700E0FFC394305003020945EFD394374003B8
:10086700020945900019E0FFC3943050030209457F
:10087700EFD39437400302094590001BE0FFC39470
:10088700305003020945EFD394374003020945303E
:100897002874900003E06435706C90004DF0A3F06D
:1008A70012EC02900078EEF0A3EFF090003D740A8E
:1008B700F0E4F55C900042E0FFE55CC39F502790B1
:1008C7000078E475F00112AB6DAFF0FE90003DE0EB
:1008D700FD04F074032DF582E43400F583E0FD1286
:1008E700C94E055C80CE90004EE004F07006900083
:1008F7004DE004F0C390004EE094E790004DE09483
:1009070003409D024425E4F55C900042E0FFE55C6E
:10091700C39F5027900078E475F00112AB6DAFF0DC
:10092700FE90003DE0FD04F074032DF582E43400F1
:10093700F583E0FD12C94E055C80CE024425900088
:100947000DE064306003020AC3A3E064376003026A
:100957000AC390001CE064206003020AC3900014DD
:10096700E0FFC394305003020AC3EFD3943340032C
:10097700020AC3900016E0FFC394305003020AC373
:10098700EFD394334003020AC3900018E0FFC394E7
:10099700305003020AC3EFD394334003020AC390D3
:1009A700001AE0FFC394305003020AC3EFD3943315
:1009B7004003020AC3900015E0FFC39430500302BE
:1009C7000AC3EFD394394003020AC3900017E0FF2C
:1009D700C394305003020AC3EFD394394003020A89
:1009E700C3900019E0FFC394305003020AC3EFD34A
:1009F70094394003020AC390001BE0FFC3943050B0
:100A070003020AC3EFD394394003020AC3302874A0
:100A1700900003E06435706C90004DF0A3F012EC89
:100A270002900078EEF0A3EFF090003D740AF0E436
:100A3700F55C900042E0FFE55CC39F50279000788B
:100A4700E475F00112AB6DAFF0FE90003DE0FD04E0
:100A5700F074032DF582E43400F583E0FD12C94EEE
:100A6700055C80CE90004EE004F0700690004DE0EB
:100A770004F0C390004EE094E790004DE0940340EB
:100A87009D024425E4F55C900042E0FFE55CC39FCE
:100A97005027900078E475F00112AB6DAFF0FE902F
:100AA700003DE0FD04F074032DF582E43400F58386
:100AB700E0FD12C94E055C80CE02442590000DE092
:100AC70064306003020FCBA3E064386003020FCBEE
:100AD700900019E064206003020FCB900018E0FF3C
:100AE70064207003020C02900014E0FEC39430509F
:100AF70003020FCBEED394394003020FCBA3E0FEE2
:100B0700C394305003020FCBEED394394003020F46
:100B1700CBA3E0FEC394305003020FCBEED394393E
:100B27004003020FCBA3E0FEC394305003020FCB68
:100B3700EED394394003020FCBEFC3943050030236
:100B47000FCBA3E0D394394003020FCB3028749026
:100B57000003E06435706C90004DF0A3F012EC02D6
:100B6700900078EEF0A3EFF090003D740AF0E4F502
:100B77005C900042E0FFE55CC39F5027900078E45B
:100B870075F00112AB6DAFF0FE90003DE0FD04F093
:100B970074032DF582E43400F583E0FD12C94E0598
:100BA7005C80CE90004EE004F0700690004DE004AB
:100BB700F0C390004EE094E790004DE09403409D11
:100BC700024425E4F55C900042E0FFE55CC39F50DA
:100BD70027900078E475F00112AB6DAFF0FE90003E
:100BE7003DE0FD04F074032DF582E43400F583E065
:100BF700FD12C94E055C80CE024425900017E0FF28
:100C070064207003020D0E900014E0FEC394305070
:100C170003020FCBEED394394003020FCBA3E0FEC0
:100C2700C394305003020FCBEED394394003020F25
:100C3700CBA3E0FEC394305003020FCBEED394391D
:100C47004003020FCBEFC394305003020FCBA3E056
:100C5700D394394003020FCB302874900003E0642B
:100C670035706C90004DF0A3F012EC02900078EE16
:100C7700F0A3EFF090003D740AF0E4F55C900042B9
:100C8700E0FFE55CC39F5027900078E475F0011200
:100C9700AB6DAFF0FE90003DE0FD04F074032DF561
:100CA70082E43400F583E0FD12C94E055C80CE90E6
:100CB700004EE004F0700690004DE004F0C3900091
:100CC7004EE094E790004DE09403409D024425E4F4
:100CD700F55C900042E0FFE55CC39F5027900078E9
:100CE700E475F00112AB6DAFF0FE90003DE0FD043E
:100CF700F074032DF582E43400F583E0FD12C94E4C
:100D0700055C80CE024425900016E0FF6420700346
:100D1700020E06900014E0FEC394305003020FCB7E
:100D2700EED394394003020FCBA3E0FEC3943050B7
:100D370003020FCBEED394394003020FCBEFC394DA
:100D4700305003020FCBA3E0D394394003020FCBFB
:100D5700302874900003E06435706C90004DF0A368
:100D6700F012EC02900078EEF0A3EFF090003D74E3
:100D77000AF0E4F55C900042E0FFE55CC39F502772
:100D8700900078E475F00112AB6DAFF0FE90003D76
:100D9700E0FD04F074032DF582E43400F583E0FDF3
:100DA70012C94E055C80CE90004EE004F0700690AC
:100DB700004DE004F0C390004EE094E790004DE052
:100DC7009403409D024425E4F55C900042E0FFE572
:100DD7005CC39F5027900078E475F00112AB6DAFAC
:100DE700F0FE90003DE0FD04F074032DF582E4343D
:100DF70000F583E0FD12C94E055C80CE02442590C4
:100E07000015E0FF64207003020EFE900014E0FE60
:100E1700C394305003020FCBEED394394003020F33
:100E2700CBEFC394305003020FCBA3E0D3943940E8
:100E370003020FCBA3E0FFC394305003020FCBEFA5
:100E4700D394394003020FCB302874900003E06439
:100E570035706C90004DF0A3F012EC02900078EE24
:100E6700F0A3EFF090003D740AF0E4F55C900042C7
:100E7700E0FFE55CC39F5027900078E475F001120E
:100E8700AB6DAFF0FE90003DE0FD04F074032DF56F
:100E970082E43400F583E0FD12C94E055C80CE90F4
:100EA700004EE004F0700690004DE004F0C390009F
:100EB7004EE094E790004DE09403409D024425E402
:100EC700F55C900042E0FFE55CC39F5027900078F7
:100ED700E475F00112AB6DAFF0FE90003DE0FD044C
:100EE700F074032DF582E43400F583E0FD12C94E5A
:100EF700055C80CE024425900014E0FF6420700357
:100F0700020FCBEFC394305003020FCBEFD39439CA
:100F17004003020FCB302874900003E06435706CF7
:100F270090004DF0A3F012EC02900078EEF0A3EFE2
:100F3700F090003D740AF0E4F55C900042E0FFE5B4
:100F47005CC39F5027900078E475F00112AB6DAF3A
:100F5700F0FE90003DE0FD04F074032DF582E434CB
:100F670000F583E0FD12C94E055C80CE90004EE08F
:100F770004F0700690004DE004F0C390004EE0943A
:100F8700E790004DE09403409D024425E4F55C9012
:100F97000042E0FFE55CC39F5027900078E475F0BE
:100FA7000112AB6DAFF0FE90003DE0FD04F074035D
:100FB7002DF582E43400F583E0FD12C94E055C800F
:100FC700CE02442590000DE0643060030214D3A3E1
:100FD700E0643960030214D3900019E064206003D1
:100FE7000214D3900018E0FF6420700302110A90E6
:100FF7000014E0FEC3943050030214D3EED39439A7
:1010070040030214D3A3E0FEC3943050030214D369
:10101700EED3943940030214D3A3E0FEC3943050B7
:10102700030214D3EED3943940030214D3A3E0FE92
:10103700C3943050030214D3EED3943940030214FF
:10104700D3EFC3943050030214D3A3E0D3943940B1
:10105700030214D3302874900003E06435706C9059
:10106700004DF0A3F012EC02900078EEF0A3EFF041
:1010770090003D740AF0E4F55C900042E0FFE55C07
:10108700C39F5027900078E475F00112AB6DAFF065
:10109700FE90003DE0FD04F074032DF582E434007A
:1010A700F583E0FD12C94E055C80CE90004EE0044A
:1010B700F0700690004DE004F0C390004EE094E716
:1010C70090004DE09403409D024425E4F55C9000B8
:1010D70042E0FFE55CC39F5027900078E475F0017C
:1010E70012AB6DAFF0FE90003DE0FD04F074032DF0
:1010F700F582E43400F583E0FD12C94E055C80CE2D
:10110700024425900017E0FF642070030212169036
:101117000014E0FEC3943050030214D3EED3943985
:1011270040030214D3A3E0FEC3943050030214D348
:10113700EED3943940030214D3A3E0FEC394305096
:10114700030214D3EED3943940030214D3EFC394AC
:101157003050030214D3A3E0D3943940030214D3CD
:10116700302874900003E06435706C90004DF0A354
:10117700F012EC02900078EEF0A3EFF090003D74CF
:101187000AF0E4F55C900042E0FFE55CC39F50275E
:10119700900078E475F00112AB6DAFF0FE90003D62
:1011A700E0FD04F074032DF582E43400F583E0FDDF
:1011B70012C94E055C80CE90004EE004F070069098
:1011C700004DE004F0C390004EE094E790004DE03E
:1011D7009403409D024425E4F55C900042E0FFE55E
:1011E7005CC39F5027900078E475F00112AB6DAF98
:1011F700F0FE90003DE0FD04F074032DF582E43429
:1012070000F583E0FD12C94E055C80CE02442590AF
:101217000016E0FF6420700302130E900014E0FE36
:10122700C3943050030214D3EED39439400302140D
:10123700D3A3E0FEC3943050030214D3EED3943902
:1012470040030214D3EFC3943050030214D3A3E036
:10125700D3943940030214D3302874900003E06418
:1012670035706C90004DF0A3F012EC02900078EE10
:10127700F0A3EFF090003D740AF0E4F55C900042B3
:10128700E0FFE55CC39F5027900078E475F00112FA
:10129700AB6DAFF0FE90003DE0FD04F074032DF55B
:1012A70082E43400F583E0FD12C94E055C80CE90E0
:1012B700004EE004F0700690004DE004F0C390008B
:1012C7004EE094E790004DE09403409D024425E4EE
:1012D700F55C900042E0FFE55CC39F5027900078E3
:1012E700E475F00112AB6DAFF0FE90003DE0FD0438
:1012F700F074032DF582E43400F583E0FD12C94E46
:10130700055C80CE024425900015E0FF6420700341
:10131700021406900014E0FEC3943050030214D365
:10132700EED3943940030214D3EFC3943050030231
:1013370014D3A3E0D3943940030214D3A3E0FFC32B
:10134700943050030214D3EFD3943940030214D3DB
:10135700302874900003E06435706C90004DF0A362
:10136700F012EC02900078EEF0A3EFF090003D74DD
:101377000AF0E4F55C900042E0FFE55CC39F50276C
:10138700900078E475F00112AB6DAFF0FE90003D70
:10139700E0FD04F074032DF582E43400F583E0FDED
:1013A70012C94E055C80CE90004EE004F0700690A6
:1013B700004DE004F0C390004EE094E790004DE04C
:1013C7009403409D024425E4F55C900042E0FFE56C
:1013D7005CC39F5027900078E475F00112AB6DAFA6
:1013E700F0FE90003DE0FD04F074032DF582E43437
:1013F70000F583E0FD12C94E055C80CE02442590BE
:101407000014E0FF642070030214D3EFC39430503C
:10141700030214D3EFD3943940030214D330287452
:10142700900003E06435706C90004DF0A3F012EC6F
:1014370002900078EEF0A3EFF090003D740AF0E41C
:10144700F55C900042E0FFE55CC39F502790007871
:10145700E475F00112AB6DAFF0FE90003DE0FD04C6
:10146700F074032DF582E43400F583E0FD12C94ED4
:10147700055C80CE90004EE004F0700690004DE0D1
:1014870004F0C390004EE094E790004DE0940340D1
:101497009D024425E4F55C900042E0FFE55CC39FB4
:1014A7005027900078E475F00112AB6DAFF0FE9015
:1014B700003DE0FD04F074032DF582E43400F5836C
:1014C700E0FD12C94E055C80CE02442590000DE078
:1014D700643160030219DBA3E0643060030219DBA7
:1014E700900019E0642060030219DB900018E0FF08
:1014F70064207003021612900014E0FEC39430506B
:10150700030219DBEED3943940030219DBA3E0FE93
:10151700C3943050030219DBEED394394003021908
:10152700DBA3E0FEC3943050030219DBEED39439FA
:1015370040030219DBA3E0FEC3943050030219DB1A
:10154700EED3943940030219DBEFC3943050030202
:1015570019DBA3E0D3943940030219DB30287490D8
:101567000003E06435706C90004DF0A3F012EC02BC
:10157700900078EEF0A3EFF090003D740AF0E4F5E8
:101587005C900042E0FFE55CC39F5027900078E441
:1015970075F00112AB6DAFF0FE90003DE0FD04F079
:1015A70074032DF582E43400F583E0FD12C94E057E
:1015B7005C80CE90004EE004F0700690004DE00491
:1015C700F0C390004EE094E790004DE09403409DF7
:1015D700024425E4F55C900042E0FFE55CC39F50C0
:1015E70027900078E475F00112AB6DAFF0FE900024
:1015F7003DE0FD04F074032DF582E43400F583E04B
:10160700FD12C94E055C80CE024425900017E0FF0D
:101617006420700302171E900014E0FEC39430503C
:10162700030219DBEED3943940030219DBA3E0FE72
:10163700C3943050030219DBEED3943940030219E7
:10164700DBA3E0FEC3943050030219DBEED39439D9
:1016570040030219DBEFC3943050030219DBA3E008
:10166700D3943940030219DB302874900003E064F7
:1016770035706C90004DF0A3F012EC02900078EEFC
:10168700F0A3EFF090003D740AF0E4F55C9000429F
:10169700E0FFE55CC39F5027900078E475F00112E6
:1016A700AB6DAFF0FE90003DE0FD04F074032DF547
:1016B70082E43400F583E0FD12C94E055C80CE90CC
:1016C700004EE004F0700690004DE004F0C3900077
:1016D7004EE094E790004DE09403409D024425E4DA
:1016E700F55C900042E0FFE55CC39F5027900078CF
:1016F700E475F00112AB6DAFF0FE90003DE0FD0424
:10170700F074032DF582E43400F583E0FD12C94E31
:10171700055C80CE024425900016E0FF642070032C
:10172700021816900014E0FEC3943050030219DB30
:10173700EED3943940030219DBA3E0FEC394305083
:10174700030219DBEED3943940030219DBEFC3948C
:101757003050030219DBA3E0D3943940030219DBAD
:10176700302874900003E06435706C90004DF0A34E
:10177700F012EC02900078EEF0A3EFF090003D74C9
:101787000AF0E4F55C900042E0FFE55CC39F502758
:10179700900078E475F00112AB6DAFF0FE90003D5C
:1017A700E0FD04F074032DF582E43400F583E0FDD9
:1017B70012C94E055C80CE90004EE004F070069092
:1017C700004DE004F0C390004EE094E790004DE038
:1017D7009403409D024425E4F55C900042E0FFE558
:1017E7005CC39F5027900078E475F00112AB6DAF92
:1017F700F0FE90003DE0FD04F074032DF582E43423
:1018070000F583E0FD12C94E055C80CE02442590A9
:101817000015E0FF6420700302190E900014E0FE2B
:10182700C3943050030219DBEED3943940030219F5
:10183700DBEFC3943050030219DBA3E0D3943940A4
:10184700030219DBA3E0FFC3943050030219DBEF57
:10185700D3943940030219DB302874900003E06405
:1018670035706C90004DF0A3F012EC02900078EE0A
:10187700F0A3EFF090003D740AF0E4F55C900042AD
:10188700E0FFE55CC39F5027900078E475F00112F4
:10189700AB6DAFF0FE90003DE0FD04F074032DF555
:1018A70082E43400F583E0FD12C94E055C80CE90DA
:1018B700004EE004F0700690004DE004F0C3900085
:1018C7004EE094E790004DE09403409D024425E4E8
:1018D700F55C900042E0FFE55CC39F5027900078DD
:1018E700E475F00112AB6DAFF0FE90003DE0FD0432
:1018F700F074032DF582E43400F583E0FD12C94E40
:10190700055C80CE024425900014E0FF642070033C
:101917000219DBEFC3943050030219DBEFD394397C
:1019270040030219DB302874900003E06435706CC3
:1019370090004DF0A3F012EC02900078EEF0A3EFC8
:10194700F090003D740AF0E4F55C900042E0FFE59A
:101957005CC39F5027900078E475F00112AB6DAF20
:10196700F0FE90003DE0FD04F074032DF582E434B1
:1019770000F583E0FD12C94E055C80CE90004EE075
:1019870004F0700690004DE004F0C390004EE09420
:10199700E790004DE09403409D024425E4F55C90F8
:1019A7000042E0FFE55CC39F5027900078E475F0A4
:1019B7000112AB6DAFF0FE90003DE0FD04F0740343
:1019C7002DF582E43400F583E0FD12C94E055C80F5
:1019D700CE02442590000DE064316003021EE3A3AC
:1019E700E064316003021EE3900019E064206003A5
:1019F700021EE3900018E0FF64207003021B1A9098
:101A07000014E0FEC394305003021EE3EED3943972
:101A17004003021EE3A3E0FEC394305003021EE31B
:101A2700EED394394003021EE3A3E0FEC394305083
:101A370003021EE3EED394394003021EE3A3E0FE44
:101A4700C394305003021EE3EED394394003021EC1
:101A5700E3EFC394305003021EE3A3E0D39439406D
:101A670003021EE3302874900003E06435706C9025
:101A7700004DF0A3F012EC02900078EEF0A3EFF027
:101A870090003D740AF0E4F55C900042E0FFE55CED
:101A9700C39F5027900078E475F00112AB6DAFF04B
:101AA700FE90003DE0FD04F074032DF582E4340060
:101AB700F583E0FD12C94E055C80CE90004EE00430
:101AC700F0700690004DE004F0C390004EE094E7FC
:101AD70090004DE09403409D024425E4F55C90009E
:101AE70042E0FFE55CC39F5027900078E475F00162
:101AF70012AB6DAFF0FE90003DE0FD04F074032DD6
:101B0700F582E43400F583E0FD12C94E055C80CE12
:101B1700024425900017E0FF64207003021C269002
:101B27000014E0FEC394305003021EE3EED3943951
:101B37004003021EE3A3E0FEC394305003021EE3FA
:101B4700EED394394003021EE3A3E0FEC394305062
:101B570003021EE3EED394394003021EE3EFC3945E
:101B6700305003021EE3A3E0D394394003021EE37F
:101B7700302874900003E06435706C90004DF0A33A
:101B8700F012EC02900078EEF0A3EFF090003D74B5
:101B97000AF0E4F55C900042E0FFE55CC39F502744
:101BA700900078E475F00112AB6DAFF0FE90003D48
:101BB700E0FD04F074032DF582E43400F583E0FDC5
:101BC70012C94E055C80CE90004EE004F07006907E
:101BD700004DE004F0C390004EE094E790004DE024
:101BE7009403409D024425E4F55C900042E0FFE544
:101BF7005CC39F5027900078E475F00112AB6DAF7E
:101C0700F0FE90003DE0FD04F074032DF582E4340E
:101C170000F583E0FD12C94E055C80CE0244259095
:101C27000016E0FF64207003021D1E900014E0FE02
:101C3700C394305003021EE3EED394394003021ECF
:101C4700E3A3E0FEC394305003021EE3EED39439BE
:101C57004003021EE3EFC394305003021EE3A3E0E8
:101C6700D394394003021EE3302874900003E064E4
:101C770035706C90004DF0A3F012EC02900078EEF6
:101C8700F0A3EFF090003D740AF0E4F55C90004299
:101C9700E0FFE55CC39F5027900078E475F00112E0
:101CA700AB6DAFF0FE90003DE0FD04F074032DF541
:101CB70082E43400F583E0FD12C94E055C80CE90C6
:101CC700004EE004F0700690004DE004F0C3900071
:101CD7004EE094E790004DE09403409D024425E4D4
:101CE700F55C900042E0FFE55CC39F5027900078C9
:101CF700E475F00112AB6DAFF0FE90003DE0FD041E
:101D0700F074032DF582E43400F583E0FD12C94E2B
:101D1700055C80CE024425900015E0FF6420700327
:101D2700021E16900014E0FEC394305003021EE317
:101D3700EED394394003021EE3EFC39430500302FD
:101D47001EE3A3E0D394394003021EE3A3E0FFC3DD
:101D570094305003021EE3EFD394394003021EE38D
:101D6700302874900003E06435706C90004DF0A348
:101D7700F012EC02900078EEF0A3EFF090003D74C3
:101D87000AF0E4F55C900042E0FFE55CC39F502752
:101D9700900078E475F00112AB6DAFF0FE90003D56
:101DA700E0FD04F074032DF582E43400F583E0FDD3
:101DB70012C94E055C80CE90004EE004F07006908C
:101DC700004DE004F0C390004EE094E790004DE032
:101DD7009403409D024425E4F55C900042E0FFE552
:101DE7005CC39F5027900078E475F00112AB6DAF8C
:101DF700F0FE90003DE0FD04F074032DF582E4341D
:101E070000F583E0FD12C94E055C80CE02442590A3
:101E17000014E0FF64207003021EE3EFC394305008
:101E270003021EE3EFD394394003021EE330287404
:101E3700900003E06435706C90004DF0A3F012EC55
:101E470002900078EEF0A3EFF090003D740AF0E402
:101E5700F55C900042E0FFE55CC39F502790007857
:101E6700E475F00112AB6DAFF0FE90003DE0FD04AC
:101E7700F074032DF582E43400F583E0FD12C94EBA
:101E8700055C80CE90004EE004F0700690004DE0B7
:101E970004F0C390004EE094E790004DE0940340B7
:101EA7009D024425E4F55C900042E0FFE55CC39F9A
:101EB7005027900078E475F00112AB6DAFF0FE90FB
:101EC700003DE0FD04F074032DF582E43400F58352
:101ED700E0FD12C94E055C80CE02442590000DE05E
:101EE700643160030223EBA3E0643260030223EB57
:101EF700900019E0642060030223EB900018E0FFD4
:101F070064207003022022900014E0FEC394305036
:101F1700030223EBEED3943940030223EBA3E0FE45
:101F2700C3943050030223EBEED3943940030223CA
:101F3700EBA3E0FEC3943050030223EBEED39439B6
:101F470040030223EBA3E0FEC3943050030223EBCC
:101F5700EED3943940030223EBEFC39430500302CE
:101F670023EBA3E0D3943940030223EB302874908A
:101F77000003E06435706C90004DF0A3F012EC02A2
:101F8700900078EEF0A3EFF090003D740AF0E4F5CE
:101F97005C900042E0FFE55CC39F5027900078E427
:101FA70075F00112AB6DAFF0FE90003DE0FD04F05F
:101FB70074032DF582E43400F583E0FD12C94E0564
:101FC7005C80CE90004EE004F0700690004DE00477
:101FD700F0C390004EE094E790004DE09403409DDD
:101FE700024425E4F55C900042E0FFE55CC39F50A6
:101FF70027900078E475F00112AB6DAFF0FE90000A
:102007003DE0FD04F074032DF582E43400F583E030
:10201700FD12C94E055C80CE024425900017E0FFF3
:102027006420700302212E900014E0FEC394305008
:10203700030223EBEED3943940030223EBA3E0FE24
:10204700C3943050030223EBEED3943940030223A9
:10205700EBA3E0FEC3943050030223EBEED3943995
:1020670040030223EBEFC3943050030223EBA3E0BA
:10207700D3943940030223EB302874900003E064C3
:1020870035706C90004DF0A3F012EC02900078EEE2
:10209700F0A3EFF090003D740AF0E4F55C90004285
:1020A700E0FFE55CC39F5027900078E475F00112CC
:1020B700AB6DAFF0FE90003DE0FD04F074032DF52D
:1020C70082E43400F583E0FD12C94E055C80CE90B2
:1020D700004EE004F0700690004DE004F0C390005D
:1020E7004EE094E790004DE09403409D024425E4C0
:1020F700F55C900042E0FFE55CC39F5027900078B5
:10210700E475F00112AB6DAFF0FE90003DE0FD0409
:10211700F074032DF582E43400F583E0FD12C94E17
:10212700055C80CE024425900016E0FF6420700312
:10213700022226900014E0FEC3943050030223EBE2
:10214700EED3943940030223EBA3E0FEC39430504F
:10215700030223EBEED3943940030223EBEFC3943E
:102167003050030223EBA3E0D3943940030223EB5F
:10217700302874900003E06435706C90004DF0A334
:10218700F012EC02900078EEF0A3EFF090003D74AF
:102197000AF0E4F55C900042E0FFE55CC39F50273E
:1021A700900078E475F00112AB6DAFF0FE90003D42
:1021B700E0FD04F074032DF582E43400F583E0FDBF
:1021C70012C94E055C80CE90004EE004F070069078
:1021D700004DE004F0C390004EE094E790004DE01E
:1021E7009403409D024425E4F55C900042E0FFE53E
:1021F7005CC39F5027900078E475F00112AB6DAF78
:10220700F0FE90003DE0FD04F074032DF582E43408
:1022170000F583E0FD12C94E055C80CE024425908F
:102227000015E0FF6420700302231E900014E0FEF7
:10223700C3943050030223EBEED3943940030223B7
:10224700EBEFC3943050030223EBA3E0D394394060
:10225700030223EBA3E0FFC3943050030223EBEF09
:10226700D3943940030223EB302874900003E064D1
:1022770035706C90004DF0A3F012EC02900078EEF0
:10228700F0A3EFF090003D740AF0E4F55C90004293
:10229700E0FFE55CC39F5027900078E475F00112DA
:1022A700AB6DAFF0FE90003DE0FD04F074032DF53B
:1022B70082E43400F583E0FD12C94E055C80CE90C0
:1022C700004EE004F0700690004DE004F0C390006B
:1022D7004EE094E790004DE09403409D024425E4CE
:1022E700F55C900042E0FFE55CC39F5027900078C3
:1022F700E475F00112AB6DAFF0FE90003DE0FD0418
:10230700F074032DF582E43400F583E0FD12C94E25
:10231700055C80CE024425900014E0FF6420700322
:102327000223EBEFC3943050030223EBEFD394392E
:1023370040030223EB302874900003E06435706C8F
:1023470090004DF0A3F012EC02900078EEF0A3EFAE
:10235700F090003D740AF0E4F55C900042E0FFE580
:102367005CC39F5027900078E475F00112AB6DAF06
:10237700F0FE90003DE0FD04F074032DF582E43497
:1023870000F583E0FD12C94E055C80CE90004EE05B
:1023970004F0700690004DE004F0C390004EE09406
:1023A700E790004DE09403409D024425E4F55C90DE
:1023B7000042E0FFE55CC39F5027900078E475F08A
:1023C7000112AB6DAFF0FE90003DE0FD04F0740329
:1023D7002DF582E43400F583E0FD12C94E055C80DB
:1023E700CE02442590000DE0643160030228F3A378
:1023F700E0643360030228F3900019E0642060036F
:102407000228F3900018E0FF6420700302252A9049
:102417000014E0FEC3943050030228F3EED394393E
:1024270040030228F3A3E0FEC3943050030228F3CD
:10243700EED3943940030228F3A3E0FEC39430504F
:10244700030228F3EED3943940030228F3A3E0FEF6
:10245700C3943050030228F3EED394394003022883
:10246700F3EFC3943050030228F3A3E0D394394029
:10247700030228F3302874900003E06435706C90F1
:10248700004DF0A3F012EC02900078EEF0A3EFF00D
:1024970090003D740AF0E4F55C900042E0FFE55CD3
:1024A700C39F5027900078E475F00112AB6DAFF031
:1024B700FE90003DE0FD04F074032DF582E4340046
:1024C700F583E0FD12C94E055C80CE90004EE00416
:1024D700F0700690004DE004F0C390004EE094E7E2
:1024E70090004DE09403409D024425E4F55C900084
:1024F70042E0FFE55CC39F5027900078E475F00148
:1025070012AB6DAFF0FE90003DE0FD04F074032DBB
:10251700F582E43400F583E0FD12C94E055C80CEF8
:10252700024425900017E0FF6420700302263690CE
:102537000014E0FEC3943050030228F3EED394391D
:1025470040030228F3A3E0FEC3943050030228F3AC
:10255700EED3943940030228F3A3E0FEC39430502E
:10256700030228F3EED3943940030228F3EFC39410
:102577003050030228F3A3E0D3943940030228F331
:10258700302874900003E06435706C90004DF0A320
:10259700F012EC02900078EEF0A3EFF090003D749B
:1025A7000AF0E4F55C900042E0FFE55CC39F50272A
:1025B700900078E475F00112AB6DAFF0FE90003D2E
:1025C700E0FD04F074032DF582E43400F583E0FDAB
:1025D70012C94E055C80CE90004EE004F070069064
:1025E700004DE004F0C390004EE094E790004DE00A
:1025F7009403409D024425E4F55C900042E0FFE52A
:102607005CC39F5027900078E475F00112AB6DAF63
:10261700F0FE90003DE0FD04F074032DF582E434F4
:1026270000F583E0FD12C94E055C80CE024425907B
:102637000016E0FF6420700302272E900014E0FECE
:10264700C3943050030228F3EED394394003022891
:10265700F3A3E0FEC3943050030228F3EED394397A
:1026670040030228F3EFC3943050030228F3A3E09A
:10267700D3943940030228F3302874900003E064B0
:1026870035706C90004DF0A3F012EC02900078EEDC
:10269700F0A3EFF090003D740AF0E4F55C9000427F
:1026A700E0FFE55CC39F5027900078E475F00112C6
:1026B700AB6DAFF0FE90003DE0FD04F074032DF527
:1026C70082E43400F583E0FD12C94E055C80CE90AC
:1026D700004EE004F0700690004DE004F0C3900057
:1026E7004EE094E790004DE09403409D024425E4BA
:1026F700F55C900042E0FFE55CC39F5027900078AF
:10270700E475F00112AB6DAFF0FE90003DE0FD0403
:10271700F074032DF582E43400F583E0FD12C94E11
:10272700055C80CE024425900015E0FF642070030D
:10273700022826900014E0FEC3943050030228F3C9
:10274700EED3943940030228F3EFC39430500302C9
:1027570028F3A3E0D3943940030228F3A3E0FFC38F
:10276700943050030228F3EFD3943940030228F33F
:10277700302874900003E06435706C90004DF0A32E
:10278700F012EC02900078EEF0A3EFF090003D74A9
:102797000AF0E4F55C900042E0FFE55CC39F502738
:1027A700900078E475F00112AB6DAFF0FE90003D3C
:1027B700E0FD04F074032DF582E43400F583E0FDB9
:1027C70012C94E055C80CE90004EE004F070069072
:1027D700004DE004F0C390004EE094E790004DE018
:1027E7009403409D024425E4F55C900042E0FFE538
:1027F7005CC39F5027900078E475F00112AB6DAF72
:10280700F0FE90003DE0FD04F074032DF582E43402
:1028170000F583E0FD12C94E055C80CE0244259089
:102827000014E0FF642070030228F3EFC3943050D4
:10283700030228F3EFD3943940030228F3302874B6
:10284700900003E06435706C90004DF0A3F012EC3B
:1028570002900078EEF0A3EFF090003D740AF0E4E8
:10286700F55C900042E0FFE55CC39F50279000783D
:10287700E475F00112AB6DAFF0FE90003DE0FD0492
:10288700F074032DF582E43400F583E0FD12C94EA0
:10289700055C80CE90004EE004F0700690004DE09D
:1028A70004F0C390004EE094E790004DE09403409D
:1028B7009D024425E4F55C900042E0FFE55CC39F80
:1028C7005027900078E475F00112AB6DAFF0FE90E1
:1028D700003DE0FD04F074032DF582E43400F58338
:1028E700E0FD12C94E055C80CE02442590000DE044
:1028F70064316003023063A3E06434600302306331
:1029070090001BE06420600302306390001AE0FF30
:1029170064207003022A5A900014E0FEC3943050DA
:1029270003023063EED394394003023063A3E0FE21
:10293700C394305003023063EED39439400302301E
:1029470063A3E0FEC394305003023063EED394399F
:102957004003023063A3E0FEC394305003023063A8
:10296700EED394394003023063A3E0FEC3943050A2
:1029770003023063EED394394003023063A3E0FED1
:10298700C394305003023063EED3943940030230CE
:1029970063EFC394305003023063A3E0D39439400C
:1029A70003023063302874900003E06435706C9044
:1029B700004DF0A3F012EC02900078EEF0A3EFF0D8
:1029C70090003D740AF0E4F55C900042E0FFE55C9E
:1029D700C39F5027900078E475F00112AB6DAFF0FC
:1029E700FE90003DE0FD04F074032DF582E4340011
:1029F700F583E0FD12C94E055C80CE90004EE004E1
:102A0700F0700690004DE004F0C390004EE094E7AC
:102A170090004DE09403409D024425E4F55C90004E
:102A270042E0FFE55CC39F5027900078E475F00112
:102A370012AB6DAFF0FE90003DE0FD04F074032D86
:102A4700F582E43400F583E0FD12C94E055C80CEC3
:102A5700024425900019E0FF64207003022B8E903A
:102A67000014E0FEC394305003023063EED3943970
:102A77004003023063A3E0FEC39430500302306387
:102A8700EED394394003023063A3E0FEC394305081
:102A970003023063EED394394003023063A3E0FEB0
:102AA700C394305003023063EED3943940030230AD
:102AB70063A3E0FEC394305003023063EED394392E
:102AC7004003023063EFC394305003023063A3E046
:102AD700D394394003023063302874900003E064D4
:102AE70035706C90004DF0A3F012EC02900078EE78
:102AF700F0A3EFF090003D740AF0E4F55C9000421B
:102B0700E0FFE55CC39F5027900078E475F0011261
:102B1700AB6DAFF0FE90003DE0FD04F074032DF5C2
:102B270082E43400F583E0FD12C94E055C80CE9047
:102B3700004EE004F0700690004DE004F0C39000F2
:102B47004EE094E790004DE09403409D024425E455
:102B5700F55C900042E0FFE55CC39F50279000784A
:102B6700E475F00112AB6DAFF0FE90003DE0FD049F
:102B7700F074032DF582E43400F583E0FD12C94EAD
:102B8700055C80CE024425900018E0FF64207003A6
:102B9700022CAE900014E0FEC39430500302306361
:102BA700EED394394003023063A3E0FEC394305060
:102BB70003023063EED394394003023063A3E0FE8F
:102BC700C394305003023063EED39439400302308C
:102BD70063A3E0FEC394305003023063EED394390D
:102BE7004003023063EFC394305003023063A3E025
:102BF700D394394003023063302874900003E064B3
:102C070035706C90004DF0A3F012EC02900078EE56
:102C1700F0A3EFF090003D740AF0E4F55C900042F9
:102C2700E0FFE55CC39F5027900078E475F0011240
:102C3700AB6DAFF0FE90003DE0FD04F074032DF5A1
:102C470082E43400F583E0FD12C94E055C80CE9026
:102C5700004EE004F0700690004DE004F0C39000D1
:102C67004EE094E790004DE09403409D024425E434
:102C7700F55C900042E0FFE55CC39F502790007829
:102C8700E475F00112AB6DAFF0FE90003DE0FD047E
:102C9700F074032DF582E43400F583E0FD12C94E8C
:102CA700055C80CE024425900017E0FF6420700386
:102CB700022DBA900014E0FEC39430500302306333
:102CC700EED394394003023063A3E0FEC39430503F
:102CD70003023063EED394394003023063A3E0FE6E
:102CE700C394305003023063EED39439400302306B
:102CF70063EFC394305003023063A3E0D3943940A9
:102D070003023063302874900003E06435706C90E0
:102D1700004DF0A3F012EC02900078EEF0A3EFF074
:102D270090003D740AF0E4F55C900042E0FFE55C3A
:102D3700C39F5027900078E475F00112AB6DAFF098
:102D4700FE90003DE0FD04F074032DF582E43400AD
:102D5700F583E0FD12C94E055C80CE90004EE0047D
:102D6700F0700690004DE004F0C390004EE094E749
:102D770090004DE09403409D024425E4F55C9000EB
:102D870042E0FFE55CC39F5027900078E475F001AF
:102D970012AB6DAFF0FE90003DE0FD04F074032D23
:102DA700F582E43400F583E0FD12C94E055C80CE60
:102DB700024425900016E0FF64207003022EB290B3
:102DC7000014E0FEC394305003023063EED394390D
:102DD7004003023063A3E0FEC39430500302306324
:102DE700EED394394003023063EFC39430500302AB
:102DF7003063A3E0D39439400302306330287490E2
:102E07000003E06435706C90004DF0A3F012EC0203
:102E1700900078EEF0A3EFF090003D740AF0E4F52F
:102E27005C900042E0FFE55CC39F5027900078E488
:102E370075F00112AB6DAFF0FE90003DE0FD04F0C0
:102E470074032DF582E43400F583E0FD12C94E05C5
:102E57005C80CE90004EE004F0700690004DE004D8
:102E6700F0C390004EE094E790004DE09403409D3E
:102E7700024425E4F55C900042E0FFE55CC39F5007
:102E870027900078E475F00112AB6DAFF0FE90006B
:102E97003DE0FD04F074032DF582E43400F583E092
:102EA700FD12C94E055C80CE024425900015E0FF57
:102EB70064207003022F96900014E0FEC3943050F4
:102EC70003023063EED394394003023063EFC394B7
:102ED700305003023063A3E0D394394003023063D8
:102EE700302874900003E06435706C90004DF0A3B7
:102EF700F012EC02900078EEF0A3EFF090003D7432
:102F07000AF0E4F55C900042E0FFE55CC39F5027C0
:102F1700900078E475F00112AB6DAFF0FE90003DC4
:102F2700E0FD04F074032DF582E43400F583E0FD41
:102F370012C94E055C80CE90004EE004F0700690FA
:102F4700004DE004F0C390004EE094E790004DE0A0
:102F57009403409D024425E4F55C900042E0FFE5C0
:102F67005CC39F5027900078E475F00112AB6DAFFA
:102F7700F0FE90003DE0FD04F074032DF582E4348B
:102F870000F583E0FD12C94E055C80CE0244259012
:102F97000014E0FF64207003023063EFC3943050E5
:102FA70003023063EFD3943940030230633028744F
:102FB700900003E06435706C90004DF0A3F012ECC4
:102FC70002900078EEF0A3EFF090003D740AF0E471
:102FD700F55C900042E0FFE55CC39F5027900078C6
:102FE700E475F00112AB6DAFF0FE90003DE0FD041B
:102FF700F074032DF582E43400F583E0FD12C94E29
:10300700055C80CE90004EE004F0700690004DE025
:1030170004F0C390004EE094E790004DE094034025
:103027009D024425E4F55C900042E0FFE55CC39F08
:103037005027900078E475F00112AB6DAFF0FE9069
:10304700003DE0FD04F074032DF582E43400F583C0
:10305700E0FD12C94E055C80CE02442590000DE0CC
:103067006431600302356BA3E06435600302356B9E
:10307700900019E06420600302356B900018E0FFB0
:10308700642070030231A2900014E0FEC394305014
:103097000302356BEED39439400302356BA3E0FE90
:1030A700C39430500302356BEED394394003023595
:1030B7006BA3E0FEC39430500302356BEED3943913
:1030C700400302356BA3E0FEC39430500302356B17
:1030D700EED39439400302356BEFC39430500302AB
:1030E700356BA3E0D39439400302356B30287490D5
:1030F7000003E06435706C90004DF0A3F012EC0211
:10310700900078EEF0A3EFF090003D740AF0E4F53C
:103117005C900042E0FFE55CC39F5027900078E495
:1031270075F00112AB6DAFF0FE90003DE0FD04F0CD
:1031370074032DF582E43400F583E0FD12C94E05D2
:103147005C80CE90004EE004F0700690004DE004E5
:10315700F0C390004EE094E790004DE09403409D4B
:10316700024425E4F55C900042E0FFE55CC39F5014
:1031770027900078E475F00112AB6DAFF0FE900078
:103187003DE0FD04F074032DF582E43400F583E09F
:10319700FD12C94E055C80CE024425900017E0FF62
:1031A700642070030232AE900014E0FEC3943050E6
:1031B7000302356BEED39439400302356BA3E0FE6F
:1031C700C39430500302356BEED394394003023574
:1031D7006BA3E0FEC39430500302356BEED39439F2
:1031E700400302356BEFC39430500302356BA3E005
:1031F700D39439400302356B302874900003E064A0
:1032070035706C90004DF0A3F012EC02900078EE50
:10321700F0A3EFF090003D740AF0E4F55C900042F3
:10322700E0FFE55CC39F5027900078E475F001123A
:10323700AB6DAFF0FE90003DE0FD04F074032DF59B
:1032470082E43400F583E0FD12C94E055C80CE9020
:10325700004EE004F0700690004DE004F0C39000CB
:103267004EE094E790004DE09403409D024425E42E
:10327700F55C900042E0FFE55CC39F502790007823
:10328700E475F00112AB6DAFF0FE90003DE0FD0478
:10329700F074032DF582E43400F583E0FD12C94E86
:1032A700055C80CE024425900016E0FF6420700381
:1032B7000233A6900014E0FEC39430500302356B2E
:1032C700EED39439400302356BA3E0FEC39430502C
:1032D7000302356BEED39439400302356BEFC39489
:1032E70030500302356BA3E0D39439400302356BAA
:1032F700302874900003E06435706C90004DF0A3A3
:10330700F012EC02900078EEF0A3EFF090003D741D
:103317000AF0E4F55C900042E0FFE55CC39F5027AC
:10332700900078E475F00112AB6DAFF0FE90003DB0
:10333700E0FD04F074032DF582E43400F583E0FD2D
:1033470012C94E055C80CE90004EE004F0700690E6
:10335700004DE004F0C390004EE094E790004DE08C
:103367009403409D024425E4F55C900042E0FFE5AC
:103377005CC39F5027900078E475F00112AB6DAFE6
:10338700F0FE90003DE0FD04F074032DF582E43477
:1033970000F583E0FD12C94E055C80CE02442590FE
:1033A7000015E0FF6420700302349E900014E0FED5
:1033B700C39430500302356BEED394394003023582
:1033C7006BEFC39430500302356BA3E0D3943940BD
:1033D7000302356BA3E0FFC39430500302356BEF54
:1033E700D39439400302356B302874900003E064AE
:1033F70035706C90004DF0A3F012EC02900078EE5F
:10340700F0A3EFF090003D740AF0E4F55C90004201
:10341700E0FFE55CC39F5027900078E475F0011248
:10342700AB6DAFF0FE90003DE0FD04F074032DF5A9
:1034370082E43400F583E0FD12C94E055C80CE902E
:10344700004EE004F0700690004DE004F0C39000D9
:103457004EE094E790004DE09403409D024425E43C
:10346700F55C900042E0FFE55CC39F502790007831
:10347700E475F00112AB6DAFF0FE90003DE0FD0486
:10348700F074032DF582E43400F583E0FD12C94E94
:10349700055C80CE024425900014E0FF6420700391
:1034A70002356BEFC39430500302356BEFD3943979
:1034B700400302356B302874900003E06435706C6C
:1034C70090004DF0A3F012EC02900078EEF0A3EF1D
:1034D700F090003D740AF0E4F55C900042E0FFE5EF
:1034E7005CC39F5027900078E475F00112AB6DAF75
:1034F700F0FE90003DE0FD04F074032DF582E43406
:1035070000F583E0FD12C94E055C80CE90004EE0C9
:1035170004F0700690004DE004F0C390004EE09474
:10352700E790004DE09403409D024425E4F55C904C
:103537000042E0FFE55CC39F5027900078E475F0F8
:103547000112AB6DAFF0FE90003DE0FD04F0740397
:103557002DF582E43400F583E0FD12C94E055C8049
:10356700CE02442590000DE064316003023B93A333
:10357700E064366003023B9390001AE06420600326
:10358700023B93900019E0FF642070030236BE905F
:103597000014E0FEC394305003023B93EED39439FA
:1035A7004003023B93A3E0FEC394305003023B93D6
:1035B700EED394394003023B93A3E0FEC39430500B
:1035C70003023B93EED394394003023B93A3E0FEFF
:1035D700C394305003023B93EED394394003023B2C
:1035E70093A3E0FEC394305003023B93EED3943988
:1035F7004003023B93EFC394305003023B93A3E095
:10360700D394394003023B93302874900003E0645D
:1036170035706C90004DF0A3F012EC02900078EE3C
:10362700F0A3EFF090003D740AF0E4F55C900042DF
:10363700E0FFE55CC39F5027900078E475F0011226
:10364700AB6DAFF0FE90003DE0FD04F074032DF587
:1036570082E43400F583E0FD12C94E055C80CE900C
:10366700004EE004F0700690004DE004F0C39000B7
:103677004EE094E790004DE09403409D024425E41A
:10368700F55C900042E0FFE55CC39F50279000780F
:10369700E475F00112AB6DAFF0FE90003DE0FD0464
:1036A700F074032DF582E43400F583E0FD12C94E72
:1036B700055C80CE024425900018E0FF642070036B
:1036C7000237DE900014E0FEC394305003023B93B0
:1036D700EED394394003023B93A3E0FEC3943050EA
:1036E70003023B93EED394394003023B93A3E0FEDE
:1036F700C394305003023B93EED394394003023B0B
:1037070093A3E0FEC394305003023B93EED3943966
:103717004003023B93EFC394305003023B93A3E073
:10372700D394394003023B93302874900003E0643C
:1037370035706C90004DF0A3F012EC02900078EE1B
:10374700F0A3EFF090003D740AF0E4F55C900042BE
:10375700E0FFE55CC39F5027900078E475F0011205
:10376700AB6DAFF0FE90003DE0FD04F074032DF566
:1037770082E43400F583E0FD12C94E055C80CE90EB
:10378700004EE004F0700690004DE004F0C3900096
:103797004EE094E790004DE09403409D024425E4F9
:1037A700F55C900042E0FFE55CC39F5027900078EE
:1037B700E475F00112AB6DAFF0FE90003DE0FD0443
:1037C700F074032DF582E43400F583E0FD12C94E51
:1037D700055C80CE024425900017E0FF642070034B
:1037E7000238EA900014E0FEC394305003023B9382
:1037F700EED394394003023B93A3E0FEC3943050C9
:1038070003023B93EED394394003023B93A3E0FEBC
:10381700C394305003023B93EED394394003023BE9
:1038270093EFC394305003023B93A3E0D394394002
:1038370003023B93302874900003E06435706C906A
:10384700004DF0A3F012EC02900078EEF0A3EFF039
:1038570090003D740AF0E4F55C900042E0FFE55CFF
:10386700C39F5027900078E475F00112AB6DAFF05D
:10387700FE90003DE0FD04F074032DF582E4340072
:10388700F583E0FD12C94E055C80CE90004EE00442
:10389700F0700690004DE004F0C390004EE094E70E
:1038A70090004DE09403409D024425E4F55C9000B0
:1038B70042E0FFE55CC39F5027900078E475F00174
:1038C70012AB6DAFF0FE90003DE0FD04F074032DE8
:1038D700F582E43400F583E0FD12C94E055C80CE25
:1038E700024425900016E0FF642070030239E2903D
:1038F7000014E0FEC394305003023B93EED3943997
:103907004003023B93A3E0FEC394305003023B9372
:10391700EED394394003023B93EFC3943050030234
:103927003B93A3E0D394394003023B933028749030
:103937000003E06435706C90004DF0A3F012EC02C8
:10394700900078EEF0A3EFF090003D740AF0E4F5F4
:103957005C900042E0FFE55CC39F5027900078E44D
:1039670075F00112AB6DAFF0FE90003DE0FD04F085
:1039770074032DF582E43400F583E0FD12C94E058A
:103987005C80CE90004EE004F0700690004DE0049D
:10399700F0C390004EE094E790004DE09403409D03
:1039A700024425E4F55C900042E0FFE55CC39F50CC
:1039B70027900078E475F00112AB6DAFF0FE900030
:1039C7003DE0FD04F074032DF582E43400F583E057
:1039D700FD12C94E055C80CE024425900015E0FF1C
:1039E70064207003023AC6900014E0FEC39430507E
:1039F70003023B93EED394394003023B93EFC39406
:103A0700305003023B93A3E0D394394003023B9326
:103A1700302874900003E06435706C90004DF0A37B
:103A2700F012EC02900078EEF0A3EFF090003D74F6
:103A37000AF0E4F55C900042E0FFE55CC39F502785
:103A4700900078E475F00112AB6DAFF0FE90003D89
:103A5700E0FD04F074032DF582E43400F583E0FD06
:103A670012C94E055C80CE90004EE004F0700690BF
:103A7700004DE004F0C390004EE094E790004DE065
:103A87009403409D024425E4F55C900042E0FFE585
:103A97005CC39F5027900078E475F00112AB6DAFBF
:103AA700F0FE90003DE0FD04F074032DF582E43450
:103AB70000F583E0FD12C94E055C80CE02442590D7
:103AC7000014E0FF64207003023B93EFC39430506F
:103AD70003023B93EFD394394003023B933028749E
:103AE700900003E06435706C90004DF0A3F012EC89
:103AF70002900078EEF0A3EFF090003D740AF0E436
:103B0700F55C900042E0FFE55CC39F50279000788A
:103B1700E475F00112AB6DAFF0FE90003DE0FD04DF
:103B2700F074032DF582E43400F583E0FD12C94EED
:103B3700055C80CE90004EE004F0700690004DE0EA
:103B470004F0C390004EE094E790004DE0940340EA
:103B57009D024425E4F55C900042E0FFE55CC39FCD
:103B67005027900078E475F00112AB6DAFF0FE902E
:103B7700003DE0FD04F074032DF582E43400F58385
:103B8700E0FD12C94E055C80CE02442590000DE091
:103B970064316003024303A3E06437600302430315
:103BA70090001BE06420600302430390001AE0FFCB
:103BB70064207003023CFA900014E0FEC394305076
:103BC70003024303EED394394003024303A3E0FE09
:103BD700C394305003024303EED3943940030243A6
:103BE70003A3E0FEC394305003024303EED394399A
:103BF7004003024303A3E0FEC39430500302430390
:103C0700EED394394003024303A3E0FEC39430503C
:103C170003024303EED394394003024303A3E0FEB8
:103C2700C394305003024303EED394394003024355
:103C370003EFC394305003024303A3E0D394394006
:103C470003024303302874900003E06435706C90DE
:103C5700004DF0A3F012EC02900078EEF0A3EFF025
:103C670090003D740AF0E4F55C900042E0FFE55CEB
:103C7700C39F5027900078E475F00112AB6DAFF049
:103C8700FE90003DE0FD04F074032DF582E434005E
:103C9700F583E0FD12C94E055C80CE90004EE0042E
:103CA700F0700690004DE004F0C390004EE094E7FA
:103CB70090004DE09403409D024425E4F55C90009C
:103CC70042E0FFE55CC39F5027900078E475F00160
:103CD70012AB6DAFF0FE90003DE0FD04F074032DD4
:103CE700F582E43400F583E0FD12C94E055C80CE11
:103CF700024425900019E0FF64207003023E2E90D5
:103D07000014E0FEC394305003024303EED394390A
:103D17004003024303A3E0FEC3943050030243036E
:103D2700EED394394003024303A3E0FEC39430501B
:103D370003024303EED394394003024303A3E0FE97
:103D4700C394305003024303EED394394003024334
:103D570003A3E0FEC394305003024303EED3943928
:103D67004003024303EFC394305003024303A3E02D
:103D7700D394394003024303302874900003E0646E
:103D870035706C90004DF0A3F012EC02900078EEC5
:103D9700F0A3EFF090003D740AF0E4F55C90004268
:103DA700E0FFE55CC39F5027900078E475F00112AF
:103DB700AB6DAFF0FE90003DE0FD04F074032DF510
:103DC70082E43400F583E0FD12C94E055C80CE9095
:103DD700004EE004F0700690004DE004F0C3900040
:103DE7004EE094E790004DE09403409D024425E4A3
:103DF700F55C900042E0FFE55CC39F502790007898
:103E0700E475F00112AB6DAFF0FE90003DE0FD04EC
:103E1700F074032DF582E43400F583E0FD12C94EFA
:103E2700055C80CE024425900018E0FF64207003F3
:103E3700023F4E900014E0FEC39430500302430348
:103E4700EED394394003024303A3E0FEC3943050FA
:103E570003024303EED394394003024303A3E0FE76
:103E6700C394305003024303EED394394003024313
:103E770003A3E0FEC394305003024303EED3943907
:103E87004003024303EFC394305003024303A3E00C
:103E9700D394394003024303302874900003E0644D
:103EA70035706C90004DF0A3F012EC02900078EEA4
:103EB700F0A3EFF090003D740AF0E4F55C90004247
:103EC700E0FFE55CC39F5027900078E475F001128E
:103ED700AB6DAFF0FE90003DE0FD04F074032DF5EF
:103EE70082E43400F583E0FD12C94E055C80CE9074
:103EF700004EE004F0700690004DE004F0C390001F
:103F07004EE094E790004DE09403409D024425E481
:103F1700F55C900042E0FFE55CC39F502790007876
:103F2700E475F00112AB6DAFF0FE90003DE0FD04CB
:103F3700F074032DF582E43400F583E0FD12C94ED9
:103F4700055C80CE024425900017E0FF64207003D3
:103F570002405A900014E0FEC3943050030243031A
:103F6700EED394394003024303A3E0FEC3943050D9
:103F770003024303EED394394003024303A3E0FE55
:103F8700C394305003024303EED3943940030243F2
:103F970003EFC394305003024303A3E0D3943940A3
:103FA70003024303302874900003E06435706C907B
:103FB700004DF0A3F012EC02900078EEF0A3EFF0C2
:103FC70090003D740AF0E4F55C900042E0FFE55C88
:103FD700C39F5027900078E475F00112AB6DAFF0E6
:103FE700FE90003DE0FD04F074032DF582E43400FB
:103FF700F583E0FD12C94E055C80CE90004EE004CB
:10400700F0700690004DE004F0C390004EE094E796
:1040170090004DE09403409D024425E4F55C900038
:1040270042E0FFE55CC39F5027900078E475F001FC
:1040370012AB6DAFF0FE90003DE0FD04F074032D70
:10404700F582E43400F583E0FD12C94E055C80CEAD
:10405700024425900016E0FF64207003024152904D
:104067000014E0FEC394305003024303EED39439A7
:104077004003024303A3E0FEC3943050030243030B
:10408700EED394394003024303EFC3943050030245
:104097004303A3E0D39439400302430330287490C9
:1040A7000003E06435706C90004DF0A3F012EC0251
:1040B700900078EEF0A3EFF090003D740AF0E4F57D
:1040C7005C900042E0FFE55CC39F5027900078E4D6
:1040D70075F00112AB6DAFF0FE90003DE0FD04F00E
:1040E70074032DF582E43400F583E0FD12C94E0513
:1040F7005C80CE90004EE004F0700690004DE00426
:10410700F0C390004EE094E790004DE09403409D8B
:10411700024425E4F55C900042E0FFE55CC39F5054
:1041270027900078E475F00112AB6DAFF0FE9000B8
:104137003DE0FD04F074032DF582E43400F583E0DF
:10414700FD12C94E055C80CE024425900015E0FFA4
:1041570064207003024236900014E0FEC39430508E
:1041670003024303EED394394003024303EFC3949E
:10417700305003024303A3E0D394394003024303BF
:10418700302874900003E06435706C90004DF0A304
:10419700F012EC02900078EEF0A3EFF090003D747F
:1041A7000AF0E4F55C900042E0FFE55CC39F50270E
:1041B700900078E475F00112AB6DAFF0FE90003D12
:1041C700E0FD04F074032DF582E43400F583E0FD8F
:1041D70012C94E055C80CE90004EE004F070069048
:1041E700004DE004F0C390004EE094E790004DE0EE
:1041F7009403409D024425E4F55C900042E0FFE50E
:104207005CC39F5027900078E475F00112AB6DAF47
:10421700F0FE90003DE0FD04F074032DF582E434D8
:1042270000F583E0FD12C94E055C80CE024425905F
:104237000014E0FF64207003024303EFC39430507F
:1042470003024303EFD39439400302430330287436
:10425700900003E06435706C90004DF0A3F012EC11
:1042670002900078EEF0A3EFF090003D740AF0E4BE
:10427700F55C900042E0FFE55CC39F502790007813
:10428700E475F00112AB6DAFF0FE90003DE0FD0468
:10429700F074032DF582E43400F583E0FD12C94E76
:1042A700055C80CE90004EE004F0700690004DE073
:1042B70004F0C390004EE094E790004DE094034073
:1042C7009D024425E4F55C900042E0FFE55CC39F56
:1042D7005027900078E475F00112AB6DAFF0FE90B7
:1042E700003DE0FD04F074032DF582E43400F5830E
:1042F700E0FD12C94E055C80CE02442590000DE01A
:1043070064316003024435A3E06438600302443536
:10431700900018E064206003024435900014E0FF29
:10432700C394305003024435EFD39437400302441B
:1043370035900016E0FFC394305003024435EFD3A5
:1043470094374003024435900015E0FFC394305082
:1043570003024435EFD394394003024435900017E4
:10436700E0FFC394305003024435EFD39439400340
:10437700024435302873900003E06435706B900079
:104387004DF0A3F012EC02900078EEF0A3EFF0905E
:10439700003D740AF0E4F55C900042E0FFE55CC381
:1043A7009F5027900078E475F00112AB6DAFF0FED7
:1043B70090003DE0FD04F074032DF582E43400F530
:1043C70083E0FD12C94E055C80CE90004EE004F0FC
:1043D700700690004DE004F0C390004EE094E79023
:1043E700004DE09403409D8035E4F55C900042E089
:1043F700FFE55CC39F5027900078E475F00112AB8E
:104407006DAFF0FE90003DE0FD04F074032DF582E2
:10441700E43400F583E0FD12C94E055C80CE7BFFD6
:104427007A55799112E95290000074FEF02212E950
:084437004C90000074FAF02221
:10CFCA00900044E0FF7003302956126A1312EC02F3
:10CFDA00900078EEF0A3EFF0E4F55C900042E0FFF9
:10CFEA00E55CC39F5027900078E475F00112AB6DA1
:10CFFA00AFF0FE12C98F8F5D7423255CF582E4348D
:10D00A0000F583E55DF01269E4055C80CE302910F5
:10D01A00C229E55C04900033F090000074F0F0221D
:10D02A00900047E0FF126A1390003D740AF0D2277D
:07D03A00900000E004F02269
:10D87400302465900001E0FF900034F0C224BF2AF8
:10D88400079000007403F022900034E0FFB42308F2
:10D89400900000E004F0803DEF547FFF1269E490B3
:10D8A4000034E0547FFF90003DE0FE04F074032E4A
:10D8B400F582E43400F583EFF0900042E02409FFA0
:10D8C400E433FE90003DE0D39FEE6480F8748098CA
:09D8D4004006900000E004F0227F
:10DD880030244B900001E0FF900034F0C224BF2AF9
:10DD9800079000007403F022900034E0FFB4230BD6
:10DDA800900000E004F0E004F0801012EFE6500F5D
:10DDB800900034E090003FF0900000E004F0227BF7
:0FDDC800FF7A55797112E95290000074FAF02237
:10C6DF0020240302C77B900001E0FF900034F0C2DA
:10C6EF0024BF2A079000007403F022900034E0FF6B
:10C6FF00B4230A900000E004F0E004F02212EFE609
:10C70F00505B90003FE0540F75F00AA4FF90003487
:10C71F00E0540F2FF0E09053DD93FF900034F012B0
:10C72F0069E4900034E0FF90003DE0FE04F07403F4
:10C73F002EF582E43400F583EFF0900042E02409F7
:10C74F00FFE433FE90003DE0D39FEE6480F87480E9
:10C75F0098900000E0400304F02214F0227BFF7A4F
:0DC76F0055797112E95290000074FAF02221
:10ECD100302109900156E0F55512EE59302303E435
:10ECE100F55530220B301F0575550A8003755528DF
:07ECF100900000E004F02296
:10D6CE00E555706512B063900041E012AB8FD6FE47
:10D6DE0064D7036ED70378D70382D7038CD7089607
:10D6EE00D70DA0D712AAD717B4D71CBE0000D71FCC
:10D6FE0012EEEF801C12E9DE801712F23B8012123E
:10D70E00F23C800D12F23D800812F23E800312F2BE
:10D71E003F30210F90017AE09000E5F0900000E09C
:0AD72E0004F0229000007401F022C4
:10EFC7009000E5E0700912EE739000007401F022E2
:10DACA0030210D900156E0F55512EE59E55570FCDE
:10DADA00302207755505E55570FCE4F55C30220CDB
:10DAEA0012F05912726412F14612726430210C1249
:10DAFA00F06412726412F146127264055CE55CC34A
:10DB0A00940540D930210E90017AE09000E5F0901A
:0CDB1A0000E5E070FA9000007401F022B9
:01F2370022B4
:01F2380022B3
:01F2390022B2
:10CD670030220A201F079000007401F02230210DA5
:10CD7700900156E0F55512EE59E55570FC30220743
:10CD8700755505E55570FC30211B900112E0F52D16
:10CD970012F064E4F55C127264055CE55CC3940A06
:10CDA70040F412F14630221B900113E0F52D12F0EA
:10CDB70059E4F55C127264055CE55CC3940A40F4BF
:10CDC70012F14630210E90017AE09000E5F09000D4
:0DCDD700E5E070FA126A4BE4900000F022D3
:01F23A0022B1
:10E623003013362024339000E87464F0E548547FB7
:10E63300FF900001F030270AE54830E70512E56E48
:10E64300EFF0D224C213900001E0B423079000023C
:0AE65300E004F022E4900002F0223F
:10E65D003011362024339000E87464F0E546547F81
:10E66D00FF900001F030270AE54630E70512E56E10
:10E67D00EFF0D224C211900001E0B4230790000204
:0AE68D00E004F022E4900002F02205
:107F9300202503028145302403028145900002E03D
:107FA300F561E4F09000E87464F012F22E8F60D271
:107FB30024E560B430079000017430F022E560B42A
:107FC30031079000017431F022E560B4320790006C
:107FD300017432F022E560B433079000017433F08A
:107FE30022E560B434079000017434F022E560B4F4
:107FF30035079000017435F022E560B43607900030
:10800300017436F022E560B437079000017437F04D
:1080130022E560B438079000017438F022E560B4BB
:1080230039079000017439F022E560B42310900001
:10803300017423F0AF610561900002EFF022E56067
:10804300B42A07900001742AF022E560B441079036
:1080530000017441F022E560B442079000017442CC
:10806300F022E560B443079000017443F022E56019
:10807300B464079000017444F022202703C2242231
:10808300E560B461079000017461F022E560B462B9
:10809300079000017462F022E560B4630790000169
:1080A3007463F022E560B464079000017464F02205
:1080B300E560B465079000017465F022E560B4667D
:1080C300079000017466F022E560B4670790000131
:1080D3007467F022E560B468079000017468F022C9
:1080E300E560B469079000017469F022E560B46A41
:1080F30007900001746AF022E560B46B07900001F9
:10810300746BF022E560B46C07900001746CF0228C
:10811300E560B46D07900001746DF022E560B46E04
:1081230007900001746EF022E560B46F07900001C0
:10813300746FF022E560B470079000017470F02250
:03814300C2242231
:0BF011007F209000037420F0A3DFFCC0
:01F01C0022D1
:0FEFE600EFC394304007EFD39439500122C32278
:10D0B60090000CE0FD6420602E90000BE0540F758C
:10D0C600F00AA4FBAAF090000AE0540F75F064A4DD
:10D0D6002BFFE5F03AFEED540F7C002FFFEC3E905F
:10D0E6000074F0A3EF803190000BE0FD6420900007
:10D0F6000A601AE0540F75F00AA4FFED540F7C0085
:10D106002FFEEC35F0900074F0A3CE800BE0540FA8
:10D11600FF900074E4F0A3EFF0E024FFF0900074B9
:05D12600E034FFF022DF
:10D94500900009E0FD6420602B900008E0540F75FD
:10D95500F00AA4FBAAF0900007E0540F75F064A448
:10D965002BFFE5F03AFEED540F7C002FFFEC3E90C7
:10D975000076802E900008E0FD6420900007601A74
:10D98500E0540F75F00AA4FFED540F7C002FFEEC58
:10D9950035F0900076F0A3CEF022E0540FFF900012
:07D9A50076E4F0A3EFF0228D
:10EDA600900005E0540F75F00AA4FFA3E0540F2F5E
:10EDB600900035F0D394004006E09415500122C32C
:01EDC600222A
:10DA6D00E4FFEF75F003A424F4F582E43451F5835B
:10DA7D00E493FE900004E0FDEE6D703BEF75F00356
:10DA8D00A424F5F582E43451F583E493FE9000056A
:10DA9D00E0FDEEB50521EF75F003A424F6F582E463
:10DAAD003451F583E493FE900006E0FDEEB50507D5
:0CDABD00900036EFF0D3220FBF33A7C358
:01DAC900223A
:10DA0D00E4FF75F003EFA4248DF582E5F03452F5B3
:10DA1D0083E493FE900004E0FDEE6D703D75F00320
:10DA2D00EFA4248EF582E5F03452F583E493FE9055
:10DA3D000005E0FDEEB5052275F003EFA4248FF58A
:10DA4D0082E5F03452F583E493FE900006E0FDEE9E
:0FDA5D00B50507900037EFF0D3220FBF70A4C3B9
:01DA6C002297
:10ACB00074032FF582E43400F583E0FD643170699C
:10ACC000FE74042FF582E43400F583E0FCEE75F0A9
:10ACD00003A424F4F582E43451F583E4936C7042C8
:10ACE00074052FF582E43400F583E0FCEE75F00383
:10ACF000A424F5F582E43451F583E493B504237478
:10AD0000062FF582E43400F583E0FCEE75F003A431
:10AD100024F6F582E43451F583E493B50404EE049B
:10AD2000FF220EBE339B7F0022ED6432706DFE74F5
:10AD3000042FF582E43400F583E0FD75F003EEA402
:10AD4000248DF582E5F03452F583E4936D704574FB
:10AD5000052FF582E43400F583E0FD75F003EEA4E1
:10AD6000248EF582E5F03452F583E493B50525741D
:10AD7000062FF582E43400F583E0FD75F003EEA4C0
:10AD8000248FF582E5F03452F583E493B50505EEA2
:0DAD90002434FF220EBE70977F00227F004A
:01AD9D002293
:10AD9E0074FE2FF582E434FFF583E0FD64317069B3
:10ADAE00FE74042FF582E43400F583E0FCEE75F0BA
:10ADBE0003A424F4F582E43451F583E4936C7042D9
:10ADCE0074052FF582E43400F583E0FCEE75F00394
:10ADDE00A424F5F582E43451F583E493B504237489
:10ADEE00062FF582E43400F583E0FCEE75F003A443
:10ADFE0024F6F582E43451F583E493B50404EE04AD
:10AE0E00FF220EBE339B7F0022ED6432706DFE7406
:10AE1E00042FF582E43400F583E0FD75F003EEA413
:10AE2E00248DF582E5F03452F583E4936D7045740C
:10AE3E00052FF582E43400F583E0FD75F003EEA4F2
:10AE4E00248EF582E5F03452F583E493B50525742E
:10AE5E00062FF582E43400F583E0FD75F003EEA4D1
:10AE6E00248FF582E5F03452F583E493B50505EEB3
:0DAE7E002434FF220EBE70977F00227F005B
:01AE8B0022A4
:10CA6100EFC3943390006F50397431F0EF75F003D8
:10CA7100A424F4F582E43451F583E493900070F03A
:10CA8100EF75F003A424F5F582E43451F583E493C2
:10CA9100900071F0EF75F003A424F6F582E43451AF
:10CAA100803A7432F075F003EFA424F4F582E5F0D6
:10CAB1003451F583E493900070F075F003EFA424F2
:10CAC100F5F582E5F03451F583E493900071F0754A
:10CAD100F003EFA424F6F582E5F03451F583E493F5
:05CAE100900072F0223C
:10EF1C00900005E0540F75F00AA4FFA3E0540F2FE6
:05EF2C00900038F02206
:10ED4000900005E0540F75F00AA4FF900004E05411
:10ED50000F75F064A42FFF900006E0540F2F900071
:03ED600039F02265
:10EF3100900005E0540F75F00AA4FFA3E0540F2FD1
:05EF410090003BF022EE
:10EC020090004CE0FF7E0090004DE0FCA3E0FD127E
:10EC1200AB0690004BE02FFF90004AE03EFE9000D2
:0AEC220043E07C002FFFEC3EFE22D1
:10EF4600900045E075F010A4243FF9744435F0FABA
:05EF56007BFF02E983CE
:03F22E007F032239
:10EEEF00302108900023E0FF12F029302208900013
:07EEFF0023E0FF12F01D22C9
:10E9DE00E4F568900033E0FFE568C39F502174238F
:10E9EE002568F582E43400F583E0F569302104FFF3
:0FE9FE0012F029302205AF6912F01D056880D490
:01EA0D0022E6
:01F23B0022B0
:01F23C0022AF
:01F23D0022AE
:01F23E0022AD
:01F23F0022AC
:0CF01D0012F06F12726412F14D02726466
:0CF0290012F07A12726412F14D0272644F
